:100000000C94760B0C94C2400C9422410C94930BEC
:100010000C94930B0C94930B0C942C410C94930B19
:100020000C94930B0C9436410C94930B0C94930BFF
:100030000C94930B0C94930B0C94930B0C94930BC8
:100040000C949C410C94930B0C94930B0C94930B79
:100050000C94C2410C94E9410C9418420C94930BFB
:100060000C94930B0C94930B0C94930B0C94930B98
:100070000C94930B0C94930B0C94930B312E323401
:100080002E30300017151515151517001212121203
:10009000121212001711111714141700171111174B
:1000A0001111170015151517111111001714141738
:1000B0001111170017141417151517000000000070
:1000C0000000000084008C0094009C00A400AC00A0
:1000D000B400BC004845414400474554202F00521D
:1000E00045424F4F540D0A0052455345540D0A00E6
:1000F0004A4A59004750530054532D4E5450303102
:100100005F585858585858006E74702E6A73742E81
:100110006D666565642E61642E6A70003030302E25
:100120003030302E3030302E303030003030302E05
:100130003030302E3030302E303030003030302EF5
:100140003030302E3030302E3030300008011C017D
:100150002C013C0174079407B407D40730313233C3
:1001600034353637383941424344454600485454C3
:10017000502F312E312032303020485454500D0A47
:10018000436F6E6E656374696F6E3A20636C6F7354
:10019000650D0A436F6E74656E742D547970653AFF
:1001A00020746578742F68746D6C0D0A4361636800
:1001B000652D436F6E74726F6C3A206E6F2D6361A4
:1001C0006368650D0A436F6E74656E742D4C616EC5
:1001D00067756167653A20656E0D0A0D0A0048541F
:1001E00054502F312E3120323030204F4B0D0A43E6
:1001F0006F6E6E656374696F6E3A20636C6F7365C2
:100200000D0A436F6E74656E742D547970653A20D3
:10021000746578742F68746D6C0D0A43616368654A
:100220002D436F6E74726F6C3A206E6F2D63616335
:1002300068650D0A436F6E74656E742D4C616E6750
:10024000756167653A20656E0D0A0D0A3C21444FC1
:1002500043545950452048544D4C205055424C4928
:100260004320222D2F2F5733432F2F44544420480F
:10027000544D4C20342E3031205472616E736974A9
:10028000696F6E616C2F2F454E2220226874747046
:100290003A2F2F7777772E77332E6F72672F54523E
:1002A0002F68746D6C342F6C6F6F73652E6474647B
:1002B000223E3C48544D4C3E3C484541443E3C5413
:1002C00049544C453E54532D4E54502D534552568F
:1002D00045522053455455503C2F5449544C453EAB
:1002E0003C2F484541443E3C424F445920424743FD
:1002F0004F4C4F523D2223464646464646464622EE
:100300003E3C43454E5445523E3C423E00223E3C1C
:100310002F464F524D3E3C42523E3C464F4E54209B
:10032000434F4C4F523D22475245454E223E564187
:100330004C55452053415645443C2F464F4E543E64
:100340003C42523E00223E3C42523E3C42523E3CE7
:10035000494E50555420545950453D225355424D15
:100360004954222056414C55453D224150504C594C
:10037000223E3C2F464F524D3E004950004E4D000C
:10038000475700444E004243007A037D03800383B5
:100390000386032000240028002C00C0006401A86C
:1003A000C000FFFFFF0101A8C00101A8C0FF01A814
:1003B000C049502041444452455353005355424E86
:1003C0004554204D41534B00474154455741590036
:1003D000444E5320534552564552004144445245E1
:1003E000535300B103BC03C803D003DB034E3100F9
:1003F0004E32004E33004E3400ED03F003F303F6AB
:1004000003534552564552310053455256455232D8
:1004100000534552564552330053455256455234C7
:10042000000104090411041904400060008000A0C8
:100430000000504F574552204F4E004558544552EA
:100440004E414C2052455345540042524F574E2086
:100450004F55542052455345540057415443484446
:100460004F472054494D455220524553455400456D
:100470004E4332384A36302052454345495645208E
:100480004552524F5200415250205245515545530A
:10049000542054494D454F5554204552524F520017
:1004A00049434D50205041434B4554204348454318
:1004B0004B2053554D204552524F5200544350202B
:1004C0005041434B455420434845434B2053554DE1
:1004D000204552524F5200554450205041434B4505
:1004E0005420434845434B2053554D204552524FCD
:1004F000520049434D50204D455353414745004418
:100500004843502052454345495645204E414B28CB
:1005100052455452592900444843502052454E45B3
:1005200057414C20535441544500444843502052B5
:100530004542494E44205354415445004448435099
:100540002045585049524544205354415445004495
:100550004843502052454345495645205041434B5E
:100560004554204552524F52004E4254205245436A
:1005700045495645204552524F52004E425420465E
:100580004F524D4154204552524F52004E4254203A
:100590005041434B4554204552524F52004E425415
:1005A0002054494D45204F555428534552564552E5
:1005B0003129004E42542054494D45204F5554286E
:1005C0005345525645523229004E42542054494D0B
:1005D00045204F5554285345525645523329004E15
:1005E00042542054494D45204F55542853455256A6
:1005F0004552342900444E532054494D45204F550F
:100600005428534552564552312900444E532054E4
:10061000494D45204F55542853455256455232298D
:1006200000444E532054494D45204F5554285345BE
:1006300052564552332900444E532054494D4520CB
:100640004F5554285345525645523429004E545064
:1006500020554E53594E43524F4E495A4544004E31
:1006600054502054494D45204F5554285345525617
:1006700045523129004E54502054494D45204F5584
:1006800054285345525645523229004E5450205456
:10069000494D45204F55542853455256455233290C
:1006A000004E54502054494D45204F555428534531
:1006B000525645523429004E545020494C4C45471F
:1006C000414C20534552564552205245504C5900FA
:1006D0004E5450204C454150205345434F4E4420EA
:1006E00041444A5553540054494D4520494C4C45CA
:1006F00047414C00475053204E4D454120464F52F4
:100700004D4154204552524F52004E4D45412043D9
:100710004845434B53554D204552524F5200544982
:100720004D452044415441205245434549564520BA
:100730004552524F5200554E53594E432054494D45
:1007400045555000310432043B044A045A046F04F6
:100750008604A004BC04D704F204FF0417052A058C
:100760003C054F0569057B058C059D05B305C9054D
:10077000DF05F5050B06210637064D065F067506F3
:100780008B06A106B706D006E706F4060A071E0781
:1007900036076E772E636769006E732E6367690094
:1007A0006E622E63676900636C2E63676900656C17
:1007B0002E6367690073642E6367690066617669FA
:1007C000636F0092079907A007A707AE07B507BC9C
:1007D00007464958204E4554574F524B20534554D5
:1007E00054494E470054494D4520534552564552B1
:1007F0002053455454494E470054494D45205052CA
:100800004F564944452053455454494E4700544996
:100810004D452042524F414443415354204C4F4791
:10082000004556454E54204C4F47005359535445AC
:100830004D20494E464F4D4154494F4E00D107E59A
:1008400007F9070E0821082B084E54502041444A4E
:100850005553544D454E54204D4F44450042524F40
:100860004144434153542041444A5553544D454E0D
:1008700054204D4F4445004750532041444A55535E
:10088000544D454E54204D4F4445004A4A5920434B
:100890004C4F434B2041444A5553544D454E5420F0
:1008A0004D4F44450049085D0877088B084E4F209E
:1008B000414C41524D2854494D452053594E4352C5
:1008C0004F4E495A4544290054494D4520414C4119
:1008D000524D284E4F542053594E43524F4E495A71
:1008E0004544290054494D4520554E41444A5553ED
:1008F0005445440054494D45204F504552415449B8
:100900004F4E2054494D454F555400465552554E73
:100910004F20525443204D4F444500465552554EAA
:100920004F20475053204D4F444500555443204DD0
:100930004F44452856414C494429005554432050C2
:1009400050534F5554204D4F44452856414C49442F
:100950002900554E49564750532054494D45204E85
:100960004F2056414C4944004E4F2054494D45209C
:10097000494E50555400AD08C808E408F4080B0966
:100980001B092B093B095209680920485454502F70
:10099000003C2F413E3C42523E003F223E003C4242
:1009A000523E3C4120485245463D222E2F00545392
:1009B0002D4E54502D5345525645523C2F423E3CED
:1009C00042523E004243004954424C00223E3C42C7
:1009D000523E3C42523E494E54455256414C285399
:1009E00065632E2030206F72203E3635353334203B
:1009F00049676E6F7265293C42523E3C494E5055E4
:100A00005420545950453D225445585422204E41BB
:100A10004D453D224954424C222053495A453D22DE
:100A20003822204D41584C454E4754483D223522EE
:100A30002056414C55453D22003530223E3C2F5436
:100A4000483E3C54482057494454483D22313530B3
:100A5000223E54494D453C2F54483E3C5448205773
:100A6000494454483D22313530223E414D4F554E88
:100A7000543C2F54483E3C54482057494454483D28
:100A800022313530223E4E4F54453C2F54483E3C97
:100A90002F54523E003C2F54443E3C2F54523E00B3
:100AA0003C2F54443E3C54443E26656D73703B00DD
:100AB0003C2F54443E3C54443E42432041444A551A
:100AC0005354006D732E007365632C006F7665724E
:100AD0002039686F7572732E00444953545249424D
:100AE0005554494F4E002D2D2D2D2D3C2F54443E55
:100AF0003C54443E003C2F54443E3C54443E00266B
:100B0000656D73703B003C2F54443E3C54443E00A2
:100B10003C545220414C49474E3D2243454E54459A
:100B200052223E3C54443E004552525253540043DC
:100B30004C520050473D3100313530223E54494D32
:100B4000453C2F54483E3C54482057494454483D66
:100B500022353030223E4556454E543C2F54483EB7
:100B60003C2F54523E003C2F54443E3C2F54523EA6
:100B70000026656D73703B3C2F54443E3C54443E0C
:100B800026656D73703B002C44415441313A002C72
:100B9000434F44453A0028545950453A002C4E459D
:100BA00058543A002C434E543A00285354533A00B8
:100BB0003C2F54443E3C54443E002D2D2D2D2F2DD2
:100BC0002D2F2D2D202D2D3A2D2D3A2D2D003C543D
:100BD0005220414C49474E3D2243454E54455222F6
:100BE0003E3C54443E003C2F5441424C453E3C4226
:100BF000523E004F5045524154494E472054494DB2
:100C000045004D494E2E00484F555220004649524E
:100C10004D574152452056455253494F4E00454E7F
:100C20004332384A3630205245564953494F4E00D8
:100C30004D414320414444524553530054494D458E
:100C400020535441545553004F5045524154494F3D
:100C50004E204D4F4445004E455442494F53204E7F
:100C6000414D4500444E532053455256455200478E
:100C70004154455741592041444452455353005330
:100C800055424E4554204D41534B0049502041445C
:100C9000445245535300323030223E4954454D3C76
:100CA0002F54483E3C54482057494454483D223331
:100CB0003030223E56414C55453C2F54483E3C2F47
:100CC00054523E003C2F54443E3C2F54523E003C74
:100CD0002F54443E3C54443E003C545220414C4925
:100CE000474E3D2243454E544552223E3C54443EDD
:100CF00000222056414C55453D220022204D4158AE
:100D00004C454E4754483D2200222053495A453D08
:100D100022003C42523E3C494E50555420545950BA
:100D2000453D225445585422204E414D453D220018
:100D3000223E3C42523E003C42523E3C2F43454EF6
:100D40005445523E3C2F424F44593E3C2F48544D4F
:100D50004C3E003C42523E3C4120485245463D22DA
:100D60002E2F223E4D41494E204D454E553C2F41A0
:100D70003E3C42523E003C42523E003F455252529F
:100D80005354223E4552524F52204F46463C2F412B
:100D90003E3C42523E0026656D73703B3C4120480C
:100DA0005245463D22003F434C52223E4C4F472085
:100DB000434C4541523C2F413E003F50473D31227C
:100DC0003E5B325D3C2F413E26656D73703B3C417E
:100DD00020485245463D22003F50473D30223E5B71
:100DE000315D3C2F413E26656D73703B3C41204890
:100DF0005245463D22003C2F5441424C453E3C4228
:100E0000523E3C4120485245463D22003C2F423E46
:100E10003C42523E3C42523E3C5441424C452042B0
:100E20004F524445523D2231223E3C54523E3C54A6
:100E3000482057494454483D220022204D455448FB
:100E40004F443D22474554003C2F423E3C42523ED7
:100E50003C464F524D20414354494F4E3D22005392
:100E6000554E004D4F4E00545545005745440054D3
:100E70004855004652490053415400414955545287
:100E8000475550564E54532D4E54502D534552569F
:100E90004552303100454E4332384A3630205245B3
:100EA000563A00494E495449414C495A494E472EF9
:100EB0002E2E00494E495449414C495A4544004B55
:100EC0004559494E50555420494C4C4547414C00DA
:100ED0004D544B3333333920494E49542E2E2E0076
:100EE00043414C2052454D3A004448435020444928
:100EF0005341424C4544004448435020454E4142F2
:100F00004C4544004E545020525820454E41424CCE
:100F10004544004E54502052582044495341424CBD
:100F200045440042524F414443415354204C4F47A3
:100F3000004F5045524154494E472054494D4500B9
:100F4000475053204D4F4445205245414459004A93
:100F50004A59204D4F444520524541445900465579
:100F600052554E4F20475053204D4F444500554E4B
:100F7000495620475053204D4F444500454E43327B
:100F8000384A363020494E495445525200850E9514
:100F90000EA30EB30EBF0ED00EE00EE90EF70E0438
:100FA0000F130F230F310F400F4F0F5E0F6E0F7C8B
:100FB0000F56657273696F6E00504C454153452062
:100FC000434845434B204B455900504C4541534500
:100FD000205245534554004D41433A004448435044
:100FE000434E543A004E42432052454D3A00574139
:100FF000495420666F722054494D45205258004391
:101000004F4E4E4543542054532D4A4A59303200D6
:10101000434845434B204349524355495400504CA3
:1010200045415345205741495400434845434B20CF
:10103000434F4E4E4543544F5200B10FB90FCA0FA4
:10104000D70FDC0FE50FEE0FFF0F10101E102A1048
:1010500045585049524544200020524542494E448B
:10106000200052454E4557414C2000494E46494EBE
:10107000495459005010591062106B104A535400D3
:101080004B535400434354005554430050535400B1
:10109000484454007C108010841088108C109010EC
:1010A0002020202020202020202020202020202040
:1010B00000504F574552204F4E0045585445524E10
:1010C000414C2052455345540042524F574E204FF9
:1010D0005554205245534554005741544348444FBA
:1010E0004720524553455400454E43205243562015
:1010F0004552524F520041525020524551205449BE
:101100004D454F55540049434D502053554D2045B2
:1011100052524F52005443502053554D2045525285
:101120004F52005544502053554D204552524F5276
:101130000049434D50204D455353414745205243AC
:101140005600444843502052454345495645204E99
:10115000414B00444843502052454E4557414C00B6
:101160004448435020524542494E4400444843506D
:10117000204558504952454400444843502050436C
:1011800054204552524F52004E4254205243562052
:101190004552524F52004E425420464F524D4154F8
:1011A000204552524F52004E4254205041434B452D
:1011B00054204552524F52004E42542054494D45FE
:1011C0004F5554284E6F3129004E42542054494DFA
:1011D000454F5554284E6F3229004E4254205449F1
:1011E0004D454F5554284E6F3329004E42542054DC
:1011F000494D454F5554284E6F342900444E5320D5
:1012000054494D454F5554284E6F312900444E5393
:101210002054494D454F5554284E6F322900444EB5
:10122000532054494D454F5554284E6F332900449F
:101230004E532054494D454F5554284E6F34290084
:101240004E545020554E53594E43524F4E495A45D5
:10125000004E54502054494D454F5554284E6F313F
:1012600029004E54502054494D454F5554284E6F37
:101270003229004E54502054494D454F5554284E64
:101280006F3329004E54502054494D454F55542832
:101290004E6F3429004E545020494C4C4547414C28
:1012A000205245502E004E5450204C454150204174
:1012B000444A5553540054494D4520494C4C4547E8
:1012C000414C0047505320464F524D415420455207
:1012D000524F52004E4D45412043484B53554D20EF
:1012E0004552522E0054494D45204441544120520C
:1012F000435645525200554E53594E432054494D82
:1013000045555000A010B110BA10C910D910E810FE
:10131000F6100611151123113111421153116011EC
:101320006C11791188119611A711B811C911DA1130
:10133000EB11FC110D121E122F12401251126212EB
:10134000731284129512A612B612C312D412E512A9
:10135000F6122D2D2F2D2D202D2D3A2D2D3A2D2D00
:1013600000484F55522020204D494E2E002A2A3A3F
:101370002A2A3A2A2A002D2D3A2D2D3A2D2D0054B5
:10138000494D450D0A00444154450D0A0061646A07
:1013900075737465640076616C69640053545553C9
:1013A0000D0A00444353540D0A005A444100524D63
:1013B0004300504645432C475074707300504D54C1
:1013C0004B3030312C3331342C330024504D544BBE
:1013D0003331342C302C312C302C312C302C302C1F
:1013E000302C302C302C302C302C302C302C302C1D
:1013F000302C302C302C312C302A32390D0A00247C
:10140000504D544B3331342C302C312C302C312C6A
:10141000302C302C302C302C302C302C302C302CEC
:10142000302C302C302C302C302C302C302A3238D0
:101430000D0A004649582049502041444452455322
:101440005300464958205355424E4554204D415370
:101450004B004649582044464C5420474154455778
:1014600041590046495820444E5320534552564551
:10147000520044484350205553452F554E5553452F
:1014800000424C4F41444341535420414444522E66
:1014900000424C4F41444341535420494E54564C12
:1014A0000042434153542043414C20524543562E61
:1014B0000054494D45205A4F4E4500475053204E49
:1014C0004F444154412054494D4552004750532008
:1014D000554E53594E432054494D4552004E4D45AB
:1014E000412053454E54454E5345003150505320F2
:1014F000494E5055542045444745004E54502052C3
:10150000582054494D454F55540041444A55535471
:1015100020574944544800475053204241554420E5
:1015200052415445005155495420544F204D414992
:101530004E00331442145214631472148114911423
:10154000A114B114BB14CC14DD14EB14FB140A1554
:10155000171525154A5354285554432B393A303022
:1015600029004B5354285554432B393A3030290025
:10157000434354285554432B383A303029005554AE
:10158000432855544320303A3030290050535428D2
:101590005554432D383A3030290048445428555486
:1015A000432D393A303029005415621570157E15D7
:1015B0008C159A15907E0000907E000080700000CF
:1015C00000000000808FFFFF7081FFFF46555255DD
:1015D0004E4F282447507470732900554E49562E9B
:1015E00028244750524D432900554E49562E282451
:1015F00047505A44412900CC15DB15E91546414CAA
:101600004C204544474500524953452045444745F1
:1016100000FD15071644495341424C4500454E41D3
:10162000424C450015161D1644495341424C450095
:10163000454E41424C45284E5450204D4F4445297B
:10164000002816301620313230306270730020329C
:101650003430306270730020343830306270730080
:101660002039363030627073003139323030627078
:1016700073003338343030627073003537363030B1
:101680006270730045164E1657166016691672166C
:101690007B1657494454483A202020202073656324
:1016A0000054494D454F55543A20202020206D7359
:1016B00000544F55543A2020202020736563005475
:1016C0004F55543A202020202073656300494E5422
:1016D000455256414C3A202020202073002F3137AC
:1016E000002D2D204D454E55202D2D0011241FBEBF
:1016F000CFEFD0E1DEBFCDBF12E0A0E0B1E0EAE382
:10170000F7EC02C005900D92AC3BB107D9F71CE095
:10171000ACEBB2E001C01D92A832B107E1F70E9424
:10172000E00E0C949B630C94000080917C01882354
:1017300059F48091EA099091EB0990930B0C8093F6
:101740000A0C81E080937C010895A0E2B0E0EBEA0E
:10175000FBE00C9430620E94E81982E00E94DC4BAE
:1017600001C0A895F999FDCF86E090E065E070E0B2
:101770000E94966301C0A895F999FDCF8EE090E094
:1017800060E570E00E94966301C0A895F999FDCFCD
:101790008CE090E06AE070E80E94966301C0A89532
:1017A000F999FDCF80E290E044E651E068EA70EC00
:1017B0000E948E6301C0A895F999FDCF84E290E064
:1017C00040E05FEF6FEF7FEF0E948E6301C0A8954E
:1017D000F999FDCF88E290E041E051E068EA70ECD1
:1017E0000E948E6301C0A895F999FDCF8CE290E02C
:1017F00041E051E068EA70EC0E948E63CE010196F0
:1018000068EF70E00E94896201C0A895F999FDCF48
:10181000CE01019660E170E040E150E00E94766305
:1018200001C0A895F999FDCF8E010F5F1F4FC80128
:1018300068E071E00E948962C80160E470E040E203
:1018400050E00E94766301C0A895F999FDCF8E0102
:101850000F5F1F4FC8016CE171E00E948962C801EF
:1018600060E670E040E250E00E94766301C0A89517
:10187000F999FDCF8E010F5F1F4FC8016CE271E037
:101880000E948962C80160E870E040E250E00E9476
:10189000766301C0A895F999FDCF8E010F5F1F4FA8
:1018A000C8016CE371E00E948962C80160EA70E0DF
:1018B00040E250E00E94766301C0A895F999FDCFFF
:1018C00080EC90E04FEF51E068EA70EC0E948E638C
:1018D00001C0A895F999FDCF84EC90E060E070E03C
:1018E0000E94966301C0A895F999FDCF86EC90E01F
:1018F00060ED77E00E94966301C0A895F999FDCF4D
:1019000088EC90E068E873E10E94966301C0A895B6
:10191000F999FDCF8CE390E061E070E00E9496635E
:1019200001C0A895F999FDCF8CEC90E060E070E0E3
:101930000E94966301C0A895F999FDCF80ED90E0D3
:1019400064EB70E00E94966301C0A895F999FDCF01
:1019500082ED90E064E873E00E94966301C0A89570
:10196000F999FDCF8EE390E065EA73EC0E949663EF
:10197000A096E4E00C944C620F931F930E944D1DBF
:1019800083B180958F70873069F40E94A50B0E9407
:10199000E81983E00E94DC4B82E00E94CF4BA895BF
:1019A000FECFA895F999FDCF8EE390E00E943C63AD
:1019B000855A934C21F00E94A50B01C0A895F99976
:1019C000FDCF86E090E00E943C639C0101978E5F12
:1019D0009F4F10F025E030E020938F0401C0A895C0
:1019E000F999FDCF8EE090E00E943C6390936705EB
:1019F0008093660501978E5F9F4F40F080E590E0F1
:101A0000909367058093660501C0A895F999FDCF6D
:101A10008CE090E00E943C639C019F779093560875
:101A200080935508C90101978E5F9F4F50F084E164
:101A3000809358088CE390E0909356088093550863
:101A400010C037FF0CC08091EE099091EF0901970B
:101A500011F084E101C085E18093580802C0109222
:101A6000580880915808882309F040C080E290E02F
:101A700044E651E068EA70EC0E94FC1B60932D057F
:101A800070932E0580932F059093300584E290E0AB
:101A900040E05FEF6FEF7FEF0E94FC1B609331052A
:101AA00070933205809333059093340588E290E07B
:101AB00041E051E068EA70EC0E94FC1B6093350540
:101AC0007093360580933705909338058CE290E04B
:101AD00041E051E068EA70EC0E94FC1B6093E10970
:101AE0007093E2098093E3099093E40980E190E028
:101AF00061ED79E048EF50E00E94D91B809103012D
:101B00006AED79E00E94A53B809104016CED79E0DB
:101B10000E94A53B809105016EED79E00E94A53BF6
:101B200080ED90E00E943C632FEF8F3F920711F40D
:101B300084EB90E09093E9098093E80982ED90E0CE
:101B40000E943C634FEF8F3F940711F484E893E0C9
:101B50009093EB098093EA0980E490E064E777E0F2
:101B600048E051E00E94B61B80E690E064E977E02F
:101B70004CE151E00E94B61B80E890E064EB77E016
:101B80004CE251E00E94B61B80EA90E064ED77E001
:101B90004CE351E00E94B61B80EC90E04FEF51E027
:101BA00068EA70EC0E94FC1B6093FA077093FB07D5
:101BB0008093FC079093FD0701C0A895F999FDCF8C
:101BC00084EC90E00E943C6390931B0880931A0879
:101BD0008F5F9F4F31F410921B0810921A0801C0BA
:101BE000A895F999FDCF86EC90E00E943C63909314
:101BF00019088093180801978E5F9F4F40F080ED81
:101C000097E0909319088093180801C0A895F99956
:101C1000FDCF88EC90E00E943C6390932008809375
:101C20001F088F5F9F4F31F488E893E1909320085D
:101C300080931F081091E709012F077011F011C060
:101C4000A895F999FDCF8AEC90E00E943C6397FD3E
:101C500008C080FF06C0187F11601093E70901C01B
:101C6000A895F999FDCF8CE390E00E943C634FEF7B
:101C70008F3F940711F480E090E00230E1F420916E
:101C8000E709277C2093E709AC0147705070413089
:101C9000510511F4286004C04230510519F4206147
:101CA0002093E70983FF07C08091E7098064809350
:101CB000E70901C0A895F999FDCF8CEC90E00E944E
:101CC0003C638093F5098F3F21F41092F50901C020
:101CD000A895F999FDCF8091F509E82FF0E0EE0F76
:101CE000FF1FEE0FFF1FEC54FA4E85919591A591C1
:101CF000B4918093770190937801A0937901B09388
:101D00007A011F910F910895EF92FF920F931F9305
:101D1000E0901A08F0901B0800E010E083E591E0E5
:101D20006DE171E00E94D23EE61AF70A080B190B2A
:101D3000B701C8011F910F91FF90EF900895EF92A6
:101D4000FF920F931F93E0901C08F0901D0800274E
:101D5000F7FC0095102F81E491E06DE171E00E94A5
:101D6000D23EE61AF70A080B190BB701C8011F91FA
:101D70000F91FF90EF9008950F931F938C010E9495
:101D8000C43D005110406F717070060F171F109303
:101D90001D0800931C080C33110534F48CE390E00B
:101DA00090931D0880931C08A1E4B1E0EDE1F1E0FF
:101DB00082E101900D928150E1F71F910F910895FA
:101DC000A4E0B0E0E6EEFEE00C942262F8941092FB
:101DD00068001CBA1DBA89E88093640080E885BF5A
:101DE00085BF80BF9FEF92B980E185B918B813E035
:101DF0001BB991B980EB84B98FE787B982EC8AB9B6
:101E000088E090E00E943663609321087093220876
:101E1000809323089093240889B18073803129F43A
:101E2000119882E08093E70905C0803239F4129856
:101E30001093E70989E080937D0103C01098109208
:101E4000E70980E18CBD81E08DBD16BC92E094BDB8
:101E500083E085BD27EC27BD90936E001092B20001
:101E60009093B00084E08093B1002093B3009093EE
:101E7000700084B780FF04C081E00E94A54F13C0AA
:101E800081FF02C082E007C082FF02C083E003C07E
:101E900083FF09C084E00E94A54F81E090E0909309
:101EA000EF098093EE0914BE8CE028E130E00FB614
:101EB000F894A895209360000FBE809360007894FA
:101EC0000E94671A0E94BC0C80E58CBD8091E709D6
:101ED0008770823011F580918F04882319F484E390
:101EE00095E01FC0813019F48AE992E01AC082306F
:101EF00019F48CE491E015C0833089F0843019F432
:101F000082E590E00EC0853019F489E290E009C0C6
:101F1000863059F48BE190E004C0833089F485EA7F
:101F200090E09093C5008093C40082E08093C0004D
:101F300086E08093C20088E98093C1008091C6004A
:101F40005E9A80E190E00E94BA1A0E948B15882365
:101F500081F484E162EA7AE00E94BA140E94E819EE
:101F600081E10E94DC4B88E00E94CF4B1798A89536
:101F7000FECF0E9461180E94E81980E00E94DC4BAD
:101F800080E00E94CF4B88E061E04CE750E00E9487
:101F9000191AC090E70927E0C2220E94C11A8C01D9
:101FA0000CC0A89582E0C81619F40E94095305C018
:101FB00093E0C91611F40E9402510E94C11A801BBD
:101FC000910B805D974068F30E94E81983E0C81682
:101FD00031F48EE00E94DC4B87E00E94CF4B809171
:101FE000E70987FF0BC085E00E94DC4B89E00E9477
:101FF000CF4B8091E70988730E94985280915808CE
:102000008823F1F081E090E090935A08809359087A
:10201000A8E0B1E0EDE1F1E082E101900D928150A4
:10202000E1F780915808843119F40E94212803C0F7
:1020300086E10E94FF28882339F00E94A54F04C042
:1020400010925A081092590892E0C91649F48091EA
:10205000E70986FF02C083E007C0C092690006C09E
:1020600023E0C21631F482E0809369001CBA81E05B
:102070008DBB1092EF091092EE090E94C11A2C013B
:102080003E010894611C711C50EC352E46E0242E54
:10209000A8950E94FA21823019F40E94662009C096
:1020A000833019F40E94DA2604C0843059F50E9466
:1020B0004724182F0E941416112321F18091E7095B
:1020C00090E087709070892BD1F4163091F4809154
:1020D000F6098823A1F0A1E4B1E0EDE1F1E082E1AD
:1020E00001900D928150E1F71092CE091092F609FD
:1020F00006C01B3121F480E490E00E94BC0E812FC9
:102100000E94A54F82E0C81619F40E94095305C029
:1021100093E0C91611F40E940251F894A090060CA5
:10212000B090070C1092070C1092060C8090080CCF
:102130009090090C1092090C1092080C789421E0F0
:10214000A216B10429F081E08816910409F0F9C1C2
:10215000F8948091020C9091030CA091040CB09122
:10216000050C89839A83AB83BC837894C3010E9456
:10217000001E009721F43092060181E0AEC0AFE26C
:10218000B1E0FC0182E101900D928150E1F7809174
:102190000601803461F58091120C8823F9F4809156
:1021A000330190913401892BC9F4809131019091D0
:1021B0003201892B99F480912F0190913001892B64
:1021C00069F489819A81AB81BC810197A109B10928
:1021D00089839A83AB83BC8382E043C08091120CD5
:1021E000823009F053C081E08093120C4FC08038D8
:1021F00009F04CC08091120C882309F047C08091EF
:10220000330190913401479709F040C0809131012A
:1022100090913201CB97D1F580912F0190913001AF
:10222000CB97A1F589819A81AB81BC810196A11DD3
:10223000B11D89839A83AB83BC838091020C9091FA
:10224000030CA091040CB091050C0196A11DB11DC9
:102250008093020C9093030CA093040CB093050C94
:1022600081E08093120CC3010E94001EAFE2B1E036
:10227000FC0122E101900D922150E1F7892B31F40C
:10228000309206011092090C1092080C89819A81F3
:10229000AB81BC8120917701309178014091790127
:1022A00050917A01820F931FA41FB51F89839A83CF
:1022B000AB83BC83C3010E94001EADE1B1E0FC0111
:1022C00082E101900D928150E1F78091120C8130F2
:1022D00039F4109206011092120C80937D010AC00D
:1022E0008091120C823031F48CE390E090931E01C7
:1022F00080931D0191E0A916B10409F0CEC00E949F
:10230000591E0E942C300E94022A80911A08909136
:102310001B08892B61F18091F7099091F8090197C9
:10232000E1F40E94840E7B018C0116161706180634
:1023300019064CF10E940F33882311F00E94A54F1B
:10234000A3E5B1E0EDE1F1E082E101900D92815071
:10235000E1F782E00E943C5016C0A3E5B1E0EDE158
:10236000F1E082E101900D928150E1F709C0A3E50F
:10237000B1E0EDE1F1E082E101900D928150E1F7F1
:10238000EE24FF248701D090E70927E0D222809134
:10239000F609882361F5DD20B1F40E949F0EAB01A0
:1023A000BC0114161506160617062CF180912D0592
:1023B00090912E05A0912F05B09130050097A105B1
:1023C000B105C9F010C083E0D81689F48091140CCF
:1023D000882369F40E949F0EAB01BC0114161506F8
:1023E0001606170644F081E08093F60904C040E029
:1023F00050E060E070E08091F4098F5F8093F40911
:102400008C33A9F41092F4098091F0099091F109AC
:10241000A091F209B091F3090196A11DB11D80931D
:10242000F0099093F109A093F209B093F309809118
:10243000E509882319F40E94C94D2FC0843019F48E
:102440000E94A54C2AC0853021F592E0D91641F0B2
:1024500021E0D21629F08091F609882309F4DFC122
:1024600080E00E94C84B80911A0890911B08892B2C
:1024700061F08091F7099091F809019731F481E0BA
:10248000B801A7010E945B4C08C081E00E94C84BC4
:1024900004C0863011F40E94E94B81E08816910453
:1024A00009F04FC08091E709877029F410927D01EF
:1024B00010927C010BC0833049F0813069F50E9495
:1024C0003C5010927D0110927C0126C080911C0826
:1024D00090911D082091FF09213019F49595879559
:1024E0000BC0223049F4880F991F24E081309207F5
:1024F0001CF080E094E005C08034910514F480E481
:1025000090E00E94BC0EA1E4B1E0EDE1F1E082E1D7
:1025100001900D928150E1F71092F60980911B0114
:1025200090911C01019769F410921C0110921B01FB
:10253000A3E5B1E0EDE1F1E082E101900D9281507F
:10254000E1F78091CE098823D9F00E947D30182FC1
:102550008823E1F080518B3058F4A1E4B1E0EDE143
:10256000F1E082E101900D928150E1F70E94CE31BD
:102570001092CE091092F609812F0E94A54F06C035
:102580001092CD091092D0091092CF098091E709DD
:102590008770823080F40E946832182F882359F0A7
:1025A0001092CE091092F60980E490E00E94BC0ED1
:1025B000812F0E94A54F81E0A816B104F1F480910B
:1025C0004205882359F0809153058150809353052B
:1025D000882321F480E090E00E9409248091540532
:1025E000882359F080916505815080936505882383
:1025F00021F481E090E00E9409248091EC099091FF
:10260000ED09019711F40E94A44E1092ED09109269
:10261000EC090E94C11A84199509409708F49DC0DD
:102620000E94C11A2C010E94431B0E94521B882346
:1026300009F493C0179A9091E509843141F480918F
:10264000E609882309F089C00E947E5954C081316F
:1026500049F49F5F80911A01891708F0E4C09091B6
:10266000E609E1C0823149F48091E609981719F42E
:1026700090911A01D8C09150D6C08331A1F48091B5
:10268000E609882339F497E09093E60926E1209340
:102690001A01C9C0873079F587E18093E60996E28F
:1026A00090931A0122C0863189F48091F7099091A4
:1026B000F809019709F051C00E940F33882311F0E7
:1026C0000E94A54F82E00E943C5047C0883179F4B7
:1026D0008091E609873021F40E948F4F97E0A3C0D4
:1026E000873109F0A0C00E949A4F97E19CC08F30BB
:1026F00041F40E94671A1092E60920921A0190E0B4
:1027000092C0803151F58091E7098770823088F45A
:102710008091F609882309F580912D0590912E0569
:10272000A0912F05B09130050097A105B105A9F042
:1027300002C0833091F481E08093F6090EC0892FA6
:1027400087500E94E54C09C0873129F4892F8751B1
:102750000E94564D02C00E94A44E80917C018823A5
:1027600021F080917C01813099F481E090E0909398
:10277000F8098093F7098091E709877082508230C9
:1027800028F41092060181E08093070115981DC07E
:1027900080917C01833029F424E020937C0185E240
:1027A00008C080917C01823031F484E080937C0108
:1027B00086E20E94A54F1092F8091092F709309214
:1027C000060190E190930701159A80911A08909163
:1027D0001B08892B41F08091F7099091F809019726
:1027E00011F4149801C0149A80915808882371F04C
:1027F00080912D0590912E05A0912F05B091300567
:102800000097A105B10511F0139801C0139A0E9419
:10281000C415813011F416983BCC169A39CC80E05F
:102820000E945B4C20CE9093E5098091E6098730A9
:1028300009F08ACF84CF8EBD0DB407FEFDCF089579
:102840002C988EBD0DB407FEFDCF1EBC0DB407FE47
:10285000FDCF8EB52C9A08952C988EBD0DB407FE31
:10286000FDCF1EBC0DB407FEFDCF8EB51EBC0DB452
:1028700007FEFDCF8EB52C9A08952C98805C8EBDF6
:102880000DB407FEFDCF6EBD0DB407FEFDCF2C9A33
:1028900008950F931F93182F0E942014082F812F43
:1028A0008F5F0E942014982F802F1F910F91089501
:1028B0000F931F93182F0E942C14082F812F8F5FC6
:1028C0000E942C14982F802F1F910F9108950F9321
:1028D0001F93182F072F0E943D14812F8F5F602FA9
:1028E0000E943D141F910F9108952C9880588EBD21
:1028F0000DB407FEFDCF6EBD0DB407FEFDCF2C9AC3
:1029000008952C9880568EBD0DB407FEFDCF6EBD88
:102910000DB407FEFDCF2C9A08951F93182F8FE159
:1029200063E00E9481148FE1612F0E9475141F9152
:1029300008951F93182F82E00E948D1484E1612F67
:102940000E943D1482E161E00E943D1483E00E94F8
:102950008D148AE00E942C1480FDFBCF82E00E943F
:102960008D1482E160E00E943D1488E10E945814B9
:102970001F910895FF920F931F93F82E8B0182E011
:102980000E948D1484E16F2D0E943D1486E1B801F0
:102990000E94671483E00E948D148AE00E942C1428
:1029A00080FDFBCF1F910F91FF9008952C988AE333
:1029B0008EBD0DB407FEFDCF1EBC0DB407FEFDCFCE
:1029C0008EB52C9A08952C988AE38EBD0DB407FE1F
:1029D000FDCF1EBC0DB407FEFDCF9EB51EBC0DB4D1
:1029E00007FEFDCF8EB52C9A08952C988AE38EBDF4
:1029F0000DB407FEFDCF1EBC0DB407FEFDCF9EB586
:102A00001EBC0DB407FEFDCF8EB51EBC0DB407FE77
:102A1000FDCF7EB51EBC0DB407FEFDCF6EB52C9A62
:102A20000895FC012C988AE38EBD0DB407FEFDCFFE
:102A300020E030E008C01EBC0DB407FEFDCF8EB50F
:102A400081932F5F3F4F26173707A8F32C9A0895DD
:102A5000982F2C988AE78EBD0DB407FEFDCF9EBD42
:102A60000DB407FEFDCF2C9A0895282F2C988AE7E5
:102A70008EBD0DB407FEFDCF9EBD0DB407FEFDCF8C
:102A80002EBD0DB407FEFDCF2C9A0895282F2C984B
:102A90008AE78EBD0DB407FEFDCF9EBD0DB407FEC7
:102AA000FDCF2EBD0DB407FEFDCF7EBD0DB407FEDC
:102AB000FDCF6EBD0DB407FEFDCF2C9A0895FC012D
:102AC0002C988AE78EBD0DB407FEFDCF20E030E0E4
:102AD00008C080818EBD0DB407FEFDCF2F5F3F4F34
:102AE000319626173707A8F32C9ACB010895282F83
:102AF0002C988AE78EBD0DB407FEFDCF80E090E0F4
:102B000005C02EBD0DB407FEFDCF019686179707B1
:102B1000C0F32C9A08958FE160E00E943D1480E19B
:102B200060E070E00E94671482E16FEF7FE10E9435
:102B300067148AE06FEF7FE10E94671483E00E94D0
:102B40008D1487E067E00E943D1487E00E94201406
:102B500080FDFBCF87E062E00E9481148FE160E39B
:102B60000E9475148FE10E94201485FDFBCF80E048
:102B70000E948D1486E10E94491420E08750984FEE
:102B800009F421E0822F089581E00E94991496951E
:102B9000879596958795817008958FE10E942014FE
:102BA0008095881F8827881F0895EF92FF920F93C2
:102BB0001F938C0180E00E948D1480E00E945814C5
:102BC000F82EE92E60919704709198046A5F7F4F08
:102BD000600F711F89E1683D780710F0685D7941E9
:102BE00080E00E9467148F2D9E2D1F910F91FF9002
:102BF000EF900895EF92FF920F931F938C0180E066
:102C00000E948D1482E00E945814F82EE92E07527B
:102C1000164E82E0B8010E9467148F2D9E2D1F91E1
:102C20000F91FF90EF9008950F931F9300919904D7
:102C300010919A040150104080E00E948D148EE1A2
:102C400060E40E947514B80189E1083D180710F08E
:102C500067ED79E18CE00E9467141F910F91089550
:102C60001F93CF93DF9381E00E948D1489E10E942E
:102C70002014182F80E00E948D148EE00E942014F2
:102C8000C82FD0E081E00E948D1489E10E942014B9
:102C9000181779F78CE00E9449149F718C179D07D3
:102CA00020F49C012952364E09C0C817D90719F4DF
:102CB00027ED39E105C09C01215030402C1B3D0B14
:102CC000C901DF91CF911F910895A7E0B0E0EBE635
:102CD000F6E10C942A628C01E0909C04F0909D0433
:102CE000E80EF91E82E0B8010E94671480E00E949D
:102CF000281584E0B8010E94671486E0B7010E949D
:102D000067148FE160E80E9475148FE160E80E940B
:102D100081148CE16AE00E9481148FE168E00E94D6
:102D2000751480919B048550823008F068C000E0E3
:102D300010E08CE10E9420148A7031F40F5F1F4F65
:102D400083E0083E1807A9F78CE10E94201481FD5A
:102D500005C083E0083E180708F451C08FE168E021
:102D60000E94811480E00E9458145C0186E00E9459
:102D700058146C010894C11CD11C80E0B6010E945B
:102D800067148E010F5F1F4FC80167E070E00E945B
:102D90001115EE24F02E012F8CE10E94201481FFEA
:102DA0002AC08C8185FF27C08FE160E80E947514DE
:102DB0008FE160E80E9481148CE16AE00E94811436
:102DC0008FE168E00E9475148CE10E9420148A70E3
:102DD000D9F38FE168E00E94811480E0B6010E947F
:102DE00067148F2D902F67E070E00E941115E39417
:102DF00080E1E81689F680E0B5010E946714279605
:102E0000EAE00C944662A0E0B0E0E9E0F7E10C945F
:102E10002B62B82E282F392F6901EE24FF24870159
:102E200011C00E94D614D82F0E94D614C82FCE01EC
:102E3000A0E0B0E0E80EF91E0A1F1B1F8EEF9FEF07
:102E4000C80ED91E92E0C916D10458F7C701D8019F
:102E50009C01AD01B0FE0BC00E94D614D82FC0E07B
:102E60009E0140E050E02E0D3F1D401F511F2030BD
:102E700080E0380781E0480780E05807A0F0CA01E9
:102E800040E050E0A0E0B0E0280F391F4A1F5B1F70
:102E9000203090E0390791E0490790E0590718F099
:102EA000C90101969C01C901CDB7DEB7E9E00C94D8
:102EB00047620F931F938B010E94D515C8010E9492
:102EC00003179C0120953095C9011F910F9108951A
:102ED000EF92FF920F931F938C017B0180E00E9481
:102EE0008D140752164E80E0B8010E946714C70186
:102EF0000E9403179C0120953095C9011F910F91E5
:102F0000FF90EF900895A0E0B0E0E9E8F7E10C94BD
:102F10002C626C017B018A014115510509F444C002
:102F20004130510551F40E94D515C7010E94FA1590
:102F30000E94D6140E94281537C080E00E948D148C
:102F4000C0919704D09198042696CC0DDD1D89E19F
:102F5000C83DD80710F0C85DD94180E1BE010E948C
:102F60006714B801615070406C0F7D1F99E1683D96
:102F7000790710F0685D794182E10E94671489ED5C
:102F800099E1E80EF91E84E1B7010E9467148FE110
:102F900060E10E9481148FE160E20E9475148FE16C
:102FA0000E94201485FDFBCFCDB7DEB7E8E00C947E
:102FB00048628FE164E00E9481148DE10E94201438
:102FC00082FDFBCF8FE10E94201487FDFBCF8EE1B5
:102FD00060E20E94751408951F93182F83E00E94E9
:102FE0008D1485E1612F0E943D141F91089583E0A7
:102FF0000E948D1485E10E9420140895FC012C98F4
:103000008AE38EBD0DB407FEFDCF20E030E00AC09C
:103010001EBC0DB407FEFDCF8EB581932F5F3F4FD1
:10302000841719F02617370798F310822C9AC901D4
:1030300008950F931F93CF93DF938C01C0E0D0E0EE
:1030400003C00E94D6142196C017D107D0F3DF9198
:10305000CF911F910F910895CF93DF93EC010E94C0
:103060009062AC012C988AE78EBD0DB407FEFDCFAF
:1030700020E030E00AC0FE01E20FF31FE491EEBD54
:103080000DB407FEFDCF2F5F3F4F2417350798F390
:103090002C9ACA01DF91CF9108958EE160E20E94DF
:1030A000811480E190E00E94BA1A8DE10E94201400
:1030B00083FDFBCF80FFF9CF8FE164E00E947514A0
:1030C00008951F938EE160E20E94811480E190E0F8
:1030D0000E94BA1A5E9880E190E00E94BA1A5E9A45
:1030E00080E190E00E94BA1A1FEF2C981EBD0DB42B
:1030F00007FEFDCF2C9A80E190E00E94BA1A8DE184
:103100000E94201483FDF1CF80FFEFCF8FE160ECB0
:103110000E943D148EE160E80E943D1488E060E06A
:1031200070E00E9467148CE067ED79E10E946714FB
:103130008AE067ED79E10E94671484E068ED79E147
:103140000E94671481E00E948D1488E161EA0E9468
:103150003D1482E00E948D1480E06DE00E943D14D9
:1031600081E060E00E943D1482E062E30E943D1431
:103170008AE06EEE75E00E94671486E062E17CE012
:103180000E94671484E062E10E943D1483E060E4E1
:103190000E943D1489E06FE30E943D1483E00E9489
:1031A0008D1485E160E00E943D1484E0609100018F
:1031B0000E943D1485E0609101010E943D1482E06F
:1031C000609102010E943D1483E0609103010E941E
:1031D0003D1480E0609104010E943D1481E0609103
:1031E00005010E943D1482E10E9420148F7180939A
:1031F0009B0480E060E070E00E94BA1480E160E02F
:1032000071E00E94BA1484E162E774E00E94BA148B
:1032100080E00E948D148FE164E00E943D141F91B4
:103220000895CF93DF93EC0181E00E948D1489E132
:103230000E942014882321F40E948D1480E044C051
:1032400080E00E948D146091990470919A0480E04E
:103250000E9467148091990490919A049093980425
:103260008093970481E994E066E070E00E94111574
:10327000809192048F7180939204809194048F7155
:1032800080939404209191043091920430939A0495
:103290002093990480919304909194048F5E9540BB
:1032A00080F489E1283D380760F420FD0AC0809150
:1032B000960487FD06C08091950484FD02C087FDB9
:1032C00006C00E94611882E0DF91CF910895F894C2
:1032D0008091020C9091030CA091040CB091050C0C
:1032E00080930A0890930B08A0930C08B0930D08E4
:1032F0008091000C9091010C909313088093120818
:103300007894CE016EE070E00E94111581E0DCCF70
:1033100098B18F70907F892B88B90895469898B19D
:103320008F70907F892B88B90000449A83E090E0E9
:103330000E94BA1A449808951F93182F88B1912FAC
:1033400092959F70807F982B98B9449A83E090E083
:103350000E94BA1A449888B11F70807F812B88B967
:10336000449A83E090E00E94BA1A44981F9108950D
:10337000469A0E949C19089546980E949C190895A7
:103380000E94B81981E090E00E94BA1A0895CF9384
:10339000DF93EC0103C021960E94C0198881882325
:1033A000D1F7DF91CF91089580E10E94BC1981E0AF
:1033B00090E00E94BA1A0895882311F48CE001C0AD
:1033C0008EE00E94BC1981E090E00E94BA1A089534
:1033D00081E00E94BC1989E190E00E94BA1A089528
:1033E000662349F0613011F4805C05C0623011F44D
:1033F0008C5E01C08C5A80680E94BC1981E090E00C
:103400000E94BA1A08950F931F93042F0E94F01977
:1034100010E004C080E20E94C0191F5F1017D4F3AF
:103420001F910F910895682F80E040E10E94031AD8
:103430000895CF93DF93EA010E94F01903C00E9420
:10344000C0192196FE0184918823C9F7DF91CF919D
:1034500008950F931F938A010E94F019C8010E94DA
:10346000C7191F910F9108951F93142F0E94F019EF
:10347000812F0E94B81981E090E00E94BA1A1F9132
:1034800008950F931F93CF93DF938B01880F880FBD
:10349000880F887380640E94BC19C0E0D0E081E08E
:1034A00090E00E94BA1A81E090E00E94BA1AF801F6
:1034B000EC0FFD1FE4918E2F0E94B8192196C830A1
:1034C000D10569F7DF91CF911F910F9108951F9357
:1034D000CF93DF9388E290E00E94C91A83E00E94B4
:1034E0008E1982E490E00E94BA1A83E00E948E193D
:1034F00081E090E00E94BA1A83E00E948E1981E078
:1035000090E00E94BA1A82E00E948E1981E090E059
:103510000E94BA1A88E20E94BC1981E090E00E94E1
:10352000BA1A88E00E94BC1981E090E00E94BA1AA1
:1035300081E00E94BC1989E190E00E94BA1A86E0FD
:103540000E94BC1981E090E00E94BA1A8CE00E94AF
:10355000BC19C4ECD0E010E0FE0165917491812F9C
:103560000E94411A1F5F22961830B1F7DF91CF9168
:103570001F91089528EC00002A95E9F70197D1F7EB
:103580000895F8942091BC023091BD027894C9014D
:103590000895AC01F8942091BC023091BD0278945A
:1035A00001C0A895F8948091BC029091BD027894D6
:1035B000821B930B84179507A0F30895DC01F89400
:1035C0007894809109048823A1F0F894E09107048D
:1035D000F0E0E95FFC4F80818C93809107048F5F5E
:1035E00080930704809109048150809309047894A2
:1035F00081E00895A1E0B0E0E0E0FBE10C943062EE
:103600008E010F5F1F4F01C0A895C8010E94DE1AEE
:103610008130D1F32196E4E00C944C62A1E0B0E05B
:10362000E4E1FBE10C943262CE0101960E94DE1AC5
:10363000882321F190918A049F3740F010928E04E4
:1036400010928D0410928A0482E019C08981E92FBA
:10365000F0E0E65FFB4F8083E92FEF5FE0938A04A1
:103660008A3061F4F0E0E65FFB4F108210928A042A
:1036700010928E0410928D0481E001C080E02196AA
:10368000E2E00C944E629091C20283B1EEEBF2E064
:10369000E90FF11D80958F7080839F5F93709093E9
:1036A000C20208959091BF028091BE02982380913A
:1036B000C00298238091C102982341F1983011F4FF
:1036C00094E11DC0943011F493E119C0923011F4CB
:1036D00092E115C0913011F491E111C09C3011F4C8
:1036E00098E10DC0933011F49FE009C0993011F4B6
:1036F00090E105C09A3011F090E001C096E1809110
:10370000150C981729F09093150C03C01092150C06
:1037100090E0892F0895EF92FF920F931F93CF931C
:10372000DF93F894E090BC02F090BD02789487019A
:10373000A895F894C091BC02D091BD027894CE01B6
:10374000801B910B409718F00E94431B8E010E9432
:10375000521B882331F4CE19DF09C051D74240F300
:1037600089E1CDB7DEB7E6E00C944A620F931F9370
:10377000CF93DF939C01EB018A0101C0A895F999D1
:10378000FDCFCE01B9014FE150E00E9426631F8EAC
:103790008881992787FD90950E945962892B21F491
:1037A000CE01B8010E948962DF91CF911F910F91E4
:1037B00008950F931F93CF93DF939C01EB018A0130
:1037C00001C0A895F999FDCFCE01B9014FE050E0B5
:1037D0000E9426631F868881992787FD90950E9405
:1037E0005962892B21F4CE01B8010E948962DF91D0
:1037F000CF911F910F910895EF92FF920F931F9316
:10380000142F052FF62EE72E01C0A895F999FDCFAC
:103810000E9436639B01AC012F3F8FEF38078FEF7B
:1038200048078FEF580741F4212F302F4F2D5E2D81
:10383000C901DA019C01AD01B901CA011F910F91C3
:10384000FF90EF9008951F93CF93DF93EC010E94B8
:103850009062182F813414F580910503909106032E
:10386000019711F4A895FECF81E090E090930603B4
:103870008093050383EC92E0BE010E9489628091EF
:10388000C3028093C60011501093040381E080931B
:1038900003038091C10080668093C100DF91CF91C6
:1038A0001F9108951F93BC01FC0101900020E9F7CE
:1038B00031971E2F181B11340CF580910503909140
:1038C0000603019711F4A895FECF81E090E0909354
:1038D00006038093050383EC92E00E9402638091CB
:1038E000C3028093C60011501093040381E08093BB
:1038F00003038091C10080668093C1001F910895E9
:103900001F93482F792F162F613444F580910503BA
:1039100090910603019711F4A895FECF81E090E005
:10392000909306038093050323EC32E0E62FFF27F4
:10393000E7FDF095C901642FAF010E94C16280913B
:10394000C3028093C60011501093040381E080935A
:1039500003038091C10080668093C1001F91089588
:103960000000000008952D9A2F98000000002F9A63
:1039700090E087FF02C02D9A01C02D982F9800007B
:1039800000002F9A9F5F983011F0880FF2CF0895B2
:103990001F93CF93DF93182FEB0180919004813018
:1039A00021F4CB010E94353EEC01F8942F9A5F9AE6
:1039B00080E30E94B31C5F982F9A5F9A1F73812F38
:1039C00080640E94B31C80E0D7FF02C02D9A01C022
:1039D0002D982F98000000002F9A000000008F5FA4
:1039E000803119F0CC0FDD1FEFCF5F982D985F9AD3
:1039F000000000001E9BFECF5F985F987894DF91D7
:103A0000CF911F9108951F93CF93DF93C0E0D1E032
:103A100012E0688179812296812F0E94C81C1F5F65
:103A20001530B9F7DF91CF911F910895FF920F9351
:103A30001F93182F062FF72EBA010E94C81C812F42
:103A40008F5F602F7F2D0E94C81C1F910F91FF90E8
:103A50000895F8942F9A5F9A8F7380680E94B31C20
:103A600080E020E030E02F98000000002F9A000056
:103A70000000220F331F1E9921608F5F803199F75C
:103A8000932F5F98789480919004813021F4822F55
:103A90000E94353E9C01C90108951F93CF93DF9387
:103AA00080E00E94291D8050904419F481E08093A9
:103AB000900482E00E94291D8F5F9F4F61F012E009
:103AC000C0E0D1E0812F0E94291D8883998322962E
:103AD0001F5F1530B9F7DF91CF911F9108959F9225
:103AE000AF92BF92CF92DF92EF92FF920F931F930C
:103AF000182F042FB52EA62E972E0E94291D6C017B
:103B0000812F8F5F0E94291D7C018FEFC8168FEFD8
:103B1000D8068FEFE8068FEFF80641F4202F3B2DF3
:103B20004A2D592DC901DA016C017D01B601C70189
:103B30001F910F91FF90EF90DF90CF90BF90AF90CB
:103B40009F9008951F1D1F1E1F1E1F1F1E1F1E1F3B
:103B5000CF93DF93EC012C964AE834D06627772781
:103B600036E4AEE6B1E0532F537009F011973217E7
:103B700029F078F56A0F7B1F3395F3CF4CE022D004
:103B8000E4E4FBE330E0C8953196313011F4511193
:103B90000A94321720F4600D711D3395F4CF402D37
:103BA000439510D02150A8F0620F711D88279927E6
:103BB00048E108D015D04CE305D012D02CE302D058
:103BC0000FD00BC03A912A912417310540F00F9085
:103BD0000F906FEF7FEF8FEF9FEFDF91CF91089501
:103BE00051E2AA1B08F4A40FA7959795879577959E
:103BF00067955A95B9F7620F711D811D911D089542
:103C0000CF93DF93FC012081318142815381CC2706
:103C1000DD2757FD3CC0C6E1DCE06CE33CD0088208
:103C2000198239D00A821B8268E135D00C821D824C
:103C3000F9012C5F3F4F67E02ED00C861D869F0157
:103C4000A6E4EEE6F1E0BA2FB37009F031972E1733
:103C50003F0720F02E1B3F0BA395F3CFAA871B86AF
:103C60002E873F87E4E4FBE3AA27C8953196A1306D
:103C700011F4B1110A942015310520F020193109F1
:103C8000A395F3CFA887198623952E833F83CE0172
:103C9000DF91CF910895002470E2220F331F441F5B
:103CA000551F001C061610F0061A23957A95A9F7E1
:103CB0000895EEECF4E08281813041F480819181BD
:103CC000019791838083892B09F412823D9685E0C8
:103CD000E633F80781F70895CF92DF92EF92FF92D3
:103CE0000F931F936B017C018AE290E090939D04F7
:103CF00080939C0480E00E948D1482E06DEC7FE153
:103D00000E9467148FEF66E070E00E94771500E074
:103D100011E0C80166E070E00E945F1586E098E05F
:103D20000E94351581E090E00E94351580E098E012
:103D30000E94351586E00E94281584E00E9428150F
:103D400081E090E00E943515C80166E070E00E94B5
:103D50005F1560912D0570912E0580912F05909132
:103D600030050E94461580E066E070E00E947715FD
:103D7000C701B6010E9446158CEC9FE10E946516B2
:103D80001F910F91FF90EF90DF90CF900895EF92E9
:103D9000FF920F931F93CF93DF937B018C01E90177
:103DA000E4ECF4E020E080819181A281B3818E1562
:103DB0009F05A007B10711F4922F0DC02F5F3D960C
:103DC000283089F7CD2BF9F090912C05892F8F5F42
:103DD000877080932C058DE0989FF0011124EC539F
:103DE000FB4FEF012496DA0186E00D900992815095
:103DF000E1F7E082F1820283138380EB94E0938702
:103E0000828781E08487CDB7DEB7E6E00C944A6212
:103E1000ACE1B0E0EEE0FFE10C942862CE01019647
:103E20006CE170E00E9411158F8198850E94353EEB
:103E30004C016F85788989899A890E94393E5B0196
:103E40006C01698D7A8D8B8D9C8D0E94393E7B0132
:103E50008C0189819A810E94353E019709F071C0D9
:103E60008B819C810E94353E8050984009F069C04A
:103E700080912D0590912E05A0912F05B0913005D0
:103E8000E816F9060A071B0709F05BC0CE01439646
:103E900060E071E046E050E00E940963009709F09D
:103EA00050C0AE14BF04C006D10611F482E04AC06F
:103EB0008E01075F1F4FC601B501A80121E030E068
:103EC0000E94C71E81E088169104D9F58CE190E02C
:103ED00090939D0480939C048EE090E00E94FA15DC
:103EE00081E090E00E94351580E098E00E94351551
:103EF00086E00E94281584E00E94281582E090E068
:103F00000E94351580E091E066E070E00E945F1548
:103F100060912D0570912E0580912F0590913005AF
:103F20000E944615C80166E070E00E945F15CE0150
:103F30000F9664E070E00E945F1586E098E00E94B2
:103F4000102080E06C96ECE00C944462EF92FF92BB
:103F50000F931F93E090A404F090A5040091A60491
:103F60001091A7042091310530913205409133051D
:103F700050913405DA01C9018E299F29A02BB12B5C
:103F80008F5F9F4FAF4FBF4F49F48EE994E06FEFC3
:103F900070E046E050E00E94DC6235C080912D0563
:103FA00090912E05A0912F05B09130058E259F256B
:103FB000A027B12782239323A423B5230097A1052B
:103FC000B10511F421E009C0E0903505F090360507
:103FD000009137051091380522E0E4ECF4E0848587
:103FE000813099F480819181A281B3818E159F05E2
:103FF000A007B10751F4AEE9B4E0349686E0019031
:104000000D928150E1F720E005C03D9685E0EC324D
:10401000F80729F7822F1F910F91FF90EF900895D5
:104020000F931F938C0180919C0490919D040E9698
:1040300090939D0480939C0480E090E00E94FA1588
:104040008EE994E066E070E00E945F1580E091E008
:1040500066E070E00E945F15C8010E94351588ED8A
:1040600099E10E9465161F910F910895AEE0B0E0AE
:10407000ECE3F0E20C943162CE0101960E9411193A
:104080008823F1F0AEE9B4E0FE01379686E00190B6
:104090000D928150E1F78D859E850E94353E28E086
:1040A0008030920711F411E00CC08650984031F432
:1040B0000E94081F182F0E94141603C00E94141695
:1040C00010E0812F2E96E3E00C944D62A8E0B0E062
:1040D000ECE6F0E20C94306282E290E00E94D515AA
:1040E000CE01019668E070E00E94111589818093ED
:1040F0003C058A8180933D0560919C0470919D04EC
:1041000082E290E00E945917892B81F08AE390E0C7
:104110000E94D5150E94F51460933E0570933F05EB
:10412000809340059093410587E057C080913C05FE
:10413000883031F16D817E818F8198850E94393E72
:104140009B01AC0160933E0570933F058093400551
:104150009093410580913C05833019F40E946118C9
:104160003BC08530C9F580913D058130A9F520938C
:1041700035053093360540933705509338052CC0EC
:1041800040919C0450919D0482E290E062E270E0D4
:104190000E94831782E290E00E94FA1580E00E945C
:1041A000281580E00E94281580E090E00E943515D7
:1041B00060919C0470919D0482E290E00E946817D7
:1041C0008C0184E290E00E94FA15C8010E94351526
:1041D00081E00E944B2101C08AE02896E4E00C9423
:1041E0004C62A0E0B0E0E7EFF0E20C942B62B82E56
:1041F000EB016A01E8EBF4E0EE24FF248701308153
:1042000021813296C901A0E0B0E0E80EF91E0A1F34
:104210001B1F84E0E43CF80791F781E0B81651F4E5
:1042200080E00E948D14C752D64E80E0BE010E94ED
:10423000671403C0CE010E94D515C6010E94031762
:104240009C0140E050E02E0D3F1D401F511F2030CB
:1042500080E0380781E0480780E05807A0F0CA01F5
:1042600040E050E0A0E0B0E0280F391F4A1F5B1F7C
:10427000203080E0380781E0480780E0580718F0D8
:10428000C90101969C0120953095C901CDB7DEB7D3
:10429000E9E00C944762ACE1B0E0E1E5F1E20C94B6
:1042A0003062182F80919C0490919D0444969093C5
:1042B0009D0480939C048EE090E00E94FA1580E0BB
:1042C00095E40E94351580919C0490919D040E9474
:1042D00035158091390590913A050E94351580E099
:1042E00090E40E94351580E40E942815812F0E94D9
:1042F000281580E090E00E94351560912D057091A1
:104300002E0580912F05909130050E9446156091F1
:10431000A4047091A5048091A6049091A7040E9422
:1043200046158EE090E064E170E00E9468178C0111
:1043300088E190E00E94FA15C8010E9435150E949C
:10434000A61F882309F443C0DE011196ECE9F4E0CE
:104350009CE101900D929150E1F7823049F4609117
:10436000350570913605809137059091380508C064
:104370006091A4047091A5048091A6049091A70473
:104380000E946C1E0E9414160E94C11A8C01A895EE
:104390000E943620882311F00E9414160E94A61F46
:1043A000882311F420E008C00E94C11A801B910BE1
:1043B0008858934160F326E0ACE9B4E0FE01319601
:1043C0008CE101900D928150E1F7222329F480E0E5
:1043D00098E00E94102020E08091390590913A05E4
:1043E000019690933A0580933905822F6C96E4E00C
:1043F0000C944C62A4E1B0E0E0E0F2E20C942E6296
:104400000E943620882309F4A1C0823011F485E08F
:104410009DC08EE090E064E170E00E945917892B06
:1044200009F091C08EE090E00E94D515CE01019672
:1044300064E170E00E94111569897A898B899C89F1
:104440000E94393E7B018C0120913105309132056B
:1044500040913305509134058981682F70E0CB017C
:10446000807F90708034910509F06DC080912D059A
:1044700090912E05A0912F05B0913005E816F90610
:104480000A071B0799F02E293F29402B512B2F5F3C
:104490003F4F4F4F5F4F51F08FEFE8168FEFF80609
:1044A0008FEF08078FEF180709F04DC06F7070701D
:1044B000660F771F660F771F60933B058B819C818A
:1044C0000E94353E20913B05821B910990939D04EB
:1044D00080939C046D857E858F8598890E94393EE6
:1044E0006093A4047093A5048093A6049093A704FA
:1044F000E092A804F092A9040093AA041093AB04DC
:1045000080913B05853120F0845190E00E9419187C
:104510006091A4047091A5048091A6049091A704D1
:104520004EE954E020E030E00E94C71E8A858130C9
:1045300011F482E00BC0813111F483E007C08630B2
:1045400011F484E003C00E94141680E06496E6E053
:104550000C944A62A0E0B0E0E0EBF2E20C942D6231
:10456000D82EEB017A0184E190E0E80EF91EF0927A
:104570009D04E0929C048CEE9FEFE80EF91E82E20F
:1045800090E00E94FA158D819E810E9435158F81E1
:1045900098850E94351569857A858B859C850E9452
:1045A00046156D857E858F8598890E94461580E524
:1045B0000E9428158D2D8F730E94281584EB95E09D
:1045C0000E94351560E070E080E090E00E944615A2
:1045D00060912D0570912E0580912F0590913005E9
:1045E0000E94393E6093B8047093B9048093BA0472
:1045F0009093BB0469817A818B819C810E94393EB2
:104600006093BC047093BD048093BE049093BF0478
:104610001092C00486E08093C10480919C04909124
:104620009D040E94353E9093C3048093C204409140
:104630009C0450919D0481E062E270E00E94F120B0
:104640008C0182E390E00E94FA15C8010E943515A2
:1046500086E00E944B21682F882301F58D2D90E084
:1046600083709070892B41F089859A85AB85BC85D4
:104670000196A11DB11D0EC0E114F10479F097015E
:1046800040E050E089859A85AB85BC85820F931FF9
:10469000A41FB51F89879A87AB87BC87862FCDB7A4
:1046A000DEB7E7E00C944962A2E1B0E0EAE5F3E2AC
:1046B0000C9432622091AC043091AD04C901A0E0A9
:1046C000B0E08A839B83AC83BD838091AE049091DC
:1046D000AF049F838E83398728871A861B861C86A2
:1046E0001D868091B4049091B504A091B604B09158
:1046F000B7040196A11DB11D8E879F87A88BB98B2A
:1047000084E0BE016F5F7F4F40E050E00E94AA222C
:104710006296E2E00C944E62A8E0B0E0E2E9F3E2D7
:104720000C9428627C018091B0049091B1040E94A5
:10473000D51500E010E06E010894C11CD11C2EE6D6
:10474000A22E27E0B22EAE0CBF1C92E0892E992437
:10475000939453C0C60165E070E04AE00E94FE17E2
:10476000080F191FC60169ED70E00E948062892B55
:1047700091F4E114F10419F08AE696E002C08AE6A9
:1047800095E06BEF70E04AE00E94FE17080F191FDA
:10479000F501908232C0C60164ED70E044E050E063
:1047A0000E949962892B19F4F501808226C08981C3
:1047B0008D30E1F48A818A30C9F48091B2049091FD
:1047C000B30408171907C8F0EE0CFF1C8AE697E03F
:1047D000E80EF91E81E090E0F7019183808315C017
:1047E0000F5F1F4F0E94D6148A3039F08091B204B7
:1047F0009091B3040817190798F38091B20490912F
:10480000B3040817190708F4A5CF2896ECE00C9418
:104810004462CF93DF93EC01009719F02AE636E06B
:1048200002C02AE635E0FE01EE0FFF1FDF0143E084
:10483000AA0FBB1F4A95E1F7AE0FBF1FAE5BBA4F81
:104840001C9211961D921D921D921C921497169601
:104850001C921E92159718961C921E9217971D96E1
:104860001D921D921D921C92509780E091E0D901FB
:10487000AC011D9241505040E1F7E659F84F1182CA
:104880001082C259D84F1882DF91CF910895A6E2C5
:10489000B0E0EDE4F4E20C94246200913B0510E0FA
:1048A000025F1F4FCE01439664E170E00E94111534
:1048B0008B899C890E94353E9093AD048093AC0413
:1048C0008D899E890E94353E9093AF048093AE04FB
:1048D0006F89788D898D9A8D0E94393E6093B404DA
:1048E0007093B5048093B6049093B7042F8D2695EA
:1048F000269530E0C801820F931F9093B1048093F6
:10490000B00480919C0490919D04821B930B909322
:10491000B3048093B2046091A4047091A5048091C3
:10492000A6049091A7040E94393E6093B804709346
:10493000B9048093BA049093BB046091A804709169
:10494000A9048091AA049091AB040E94393E60931F
:10495000BC047093BD048093BE049093BF04109276
:10496000C00486E08093C10480919C0490919D04D2
:104970000E94353E9093C3048093C20440919C04EE
:1049800050919D0480E0B8010E94F120892B09F02C
:1049900099C198A1992309F495C16090A4047090DD
:1049A000A5048090A6049090A704E090AC04F09039
:1049B000AD04A090AE04B090AF0402E415E0CC24A6
:1049C000DD246FEF7FEF2E010894411C511CD201B2
:1049D000F80182E101900D928150E1F7AE81BF8133
:1049E000E885F9852A813B814C815D818981882315
:1049F00031F48FEF6F3F780711F4B6010BC0261525
:104A000037054805590531F4EE15FF0519F4AA15C7
:104A1000BB05C1F00894C11CD11C0E5E1F4FE2E023
:104A2000CE16D104A1F6FFEF6F3F7F0741F06B0177
:104A3000C094D0948CE9C8168FEFD80619F40E9460
:104A40005423FFC0D7FE47C091FF3FC18091660548
:104A500090916705A816B90609F037C1C094D094A3
:104A6000C601880F991F8C0143E0000F111F4A9562
:104A7000E1F7080F191F0E5B1A4FF801618272826D
:104A800083829482B682A582F086E78281E0808369
:104A90000E94C43DF8016187728783879487809163
:104AA000B4049091B504A091B604B091B7040196F6
:104AB000A11DB11D85879687A787B08B8CE3818B5D
:104AC00082E1B80140E050E00E94AA22F82E88233B
:104AD00009F4FCC053C091FF03C00E9454234DC091
:104AE00092FF0FC0B601660F771FCB0123E0880F3E
:104AF000991F2A95E1F7680F791F6E5B7A4F84E062
:104B000038C090FF3FC0C601880F991F8C01B3E0E9
:104B1000000F111FBA95E1F7080F191F0E5B1A4F0E
:104B2000F80120818091B4049091B504A091B6045D
:104B3000B091B7040196A11DB11D85879687A787FF
:104B4000B08B223079F480E1B80140E050E00E945F
:104B5000AA2281E1B80140E050E00E94AA22F82E8A
:104B600085E0A1C0233019F0263009F0AEC080E105
:104B7000B80140E050E00E94AA22F82EC6010E942F
:104B80000924A4C093FF5FC08091B2049091B30444
:104B9000009711F480E055C05601AA0CBB1C85019A
:104BA000F3E0000F111FFA95E1F70A0D1B1D0E5BD4
:104BB0001A4FF8012081213019F482E0808302C06D
:104BC000223011F0FF243CC0A0E0B0E02091B404FA
:104BD0003091B5044091B6045091B704820F931FF1
:104BE000A41FB51FF80185879687A787B08B2581FD
:104BF0003681809166059091670528173907B1F4D1
:104C000080E1B80140E050E00E94AA22F82EC601DF
:104C10000E948C23F501E659F84F8081918101971C
:104C200079F4C6010E941F45F82E0AC081E1B8013F
:104C300040E050E00E94AA22F82E83E0F801808331
:104C40008F2DF82E43C094FF40C0C601880F991FD6
:104C50008C0173E0000F111F7A95E1F7080F191FFF
:104C60000E5B1A4FF8018081813011F482E022C07E
:104C70008230E1F48091B2049091B304892B59F011
:104C800080E1B80140E050E00E94AA22F82EC6015F
:104C90000E948C231BC081E1B80140E050E00E94DB
:104CA000AA22F82E83E0F801808310C0833021F41B
:104CB00086E0F801808309C0853039F4C6010E947E
:104CC000092403C068E0F62E01C0FF248F2DA696AC
:104CD000E0E10C944062CF93DF93089690939D049B
:104CE00080939C0482E290E00E94FA158091AE04C9
:104CF0009091AF040E9435158091AC049091AD0461
:104D00000E94351580919C0490919D040E94351558
:104D100080E090E00E94351560912D0570912E0580
:104D200080912F05909130050E94393E6093B80420
:104D30007093B9048093BA049093BB046091A40467
:104D40007091A5048091A6049091A7040E94393E19
:104D50006093BC047093BD048093BE049093BF0421
:104D60001092C00481E18093C10480919C049091D1
:104D70009D040E94353E9093C3048093C2044091E9
:104D80009C0450919D0481E062E270E00E94F12059
:104D9000EC01009711F4CFEFDFEF88E290E00E9482
:104DA000FA15CE010E94351581E10E944B21DF9159
:104DB000CF910895A0E1B0E0E0EEF6E20C942E620F
:104DC000CE01099668E070E00E94111589859A85E8
:104DD0000E94353E9093AD048093AC048B859C85F6
:104DE0000E94353E9093AF048093AE048D859E85DE
:104DF0000E94353E8C01085010401093B30400937C
:104E0000B204085F1F4F80913B05E82EFF248EE01F
:104E100090E0E80EF91E8F859889892BB9F1609191
:104E2000A4047091A5048091A6049091A7040E9407
:104E3000393E6093B8047093B9048093BA04909398
:104E4000BB046091A8047091A9048091AA04909178
:104E5000AB040E94393E6093BC047093BD04809300
:104E6000BE049093BF041092C00481E18093C104FA
:104E70008D859E859093C3048093C20480E0B70122
:104E8000A8010E94F120892B09F04AC0C7010896A9
:104E90009093B1048093B0042091AE043091AF049C
:104EA0002B37310519F40E94C7333DC02532310537
:104EB00019F40E94843B37C044E02030340719F4D1
:104EC0000E94392D30C02434310519F40E94F92A8A
:104ED0002AC02938310519F40E94812E24C021519D
:104EE000374201F50E94D5158E010F5F1F4FC80193
:104EF00067E070E00E941115C80168EE70E047E0BD
:104F000050E00E949962892B69F48AE290E00E9445
:104F1000FA158FED90E00E942C180E946B26FFCFAF
:104F200089E001C080E06096E6E00C944A628091DE
:104F30002D0890912E08A0912F08B09130088093F1
:104F4000A4049093A504A093A604B093A70483E4BB
:104F500090E09093AD048093AC0484E490E090934F
:104F6000AF048093AE048AE290E00E94FA1560E0FC
:104F700076E081E091E00E9446150E94C43D609376
:104F800041087093420880934308909344080E941C
:104F9000461580E090E00E94351580E090E00E9488
:104FA000351560E070E080E090E00E94461580E0FA
:104FB0006CE070E00E94771580E091E066E070E0C0
:104FC0000E945F1580E06AEC70E00E94771563E64E
:104FD00073E582E893E60E94461581E095E30E941E
:104FE000351584E00E94281582E30E94281584E08C
:104FF0000E94281560912D0570912E0580912F0536
:10500000909130050E94461586E30E94281584E0A1
:105010000E94281560912D0870912E0880912F080C
:10502000909130080E9446158FEF0E94281580E06D
:105030006CE270E00E9477158CE291E00E946B2692
:1050400008950F931F9381E0809358088FEF9FEF8F
:10505000AFEFBFEF8093A4049093A504A093A604A0
:10506000B093A70483E490E09093AD048093AC04E4
:1050700084E490E09093AF048093AE0410923105E5
:1050800010923205109233051092340510922D05BE
:1050900010922E0510922F05109230051092E10902
:1050A0001092E2091092E3091092E409109235057A
:1050B0001092360510923705109238051092290883
:1050C00010922A0810922B0810922C081092250892
:1050D0001092260810922708109228081092310882
:1050E00010923208109233081092340810922D0852
:1050F00010922E0810922F081092300810923D083E
:1051000010923E0810923F08109240081092350805
:105110001092360810923708109238081092390809
:1051200010923A0810923B0810923C0810924D08D9
:1051300010924E0810924F081092500810925B087F
:105140000E94C43D609341087093420880934308D5
:10515000909344088AE290E00E94FA1560E076E0BD
:1051600081E091E00E9446156091410870914208EB
:1051700080914308909144080E94461560E070E8D1
:1051800080E090E00E94461580E060E170E00E94BF
:10519000771500E011E0C80166E070E00E945F153D
:1051A00080E06AEC70E00E94771563E673E582E8C0
:1051B00093E60E94461581E095E30E94351581E053
:1051C0000E9428158DE30E94281587E00E9428156B
:1051D00081E00E942815C80166E070E00E945F151A
:1051E0008FEF0E94281580E06FE270E00E94771533
:1051F0008CE291E00E946B261F910F9108950F930E
:105200001F93182F80935808883129F08FEF9FEF54
:10521000AFEFBFEF08C080912D0890912E08A091AC
:105220002F08B09130088093A4049093A504A09314
:10523000A604B093A704133051F00E94C43D6093BC
:105240004108709342088093430890934408E1ED2D
:10525000F9E001900020E9F73197E15DF9400E2F68
:105260000F5F83E490E09093AD048093AC0484E4FA
:1052700090E09093AF048093AE048AE290E00E94A5
:10528000FA1560E076E081E091E00E9446156091B9
:1052900041087091420880914308909144080E940F
:1052A000461580E090E00E943515183119F080E035
:1052B00090E802C080E090E00E94351560912D05D5
:1052C00070912E0580912F05909130050E94461512
:1052D00080E06CE070E00E94771580E091E066E08D
:1052E00070E00E945F1580E06AEC70E00E94771524
:1052F00063E673E582E893E60E94461581E095E354
:105300000E94351583E00E9428158CE00E94281524
:10531000802F0E94281581ED99E0602F70E00E9497
:105320005F15133019F582E30E94281584E00E946E
:1053300028158091B0049091B10440960E94D51533
:105340000E94F5140E94461586E30E94281584E009
:105350000E94281560912D0870912E0880912F08C9
:10536000909130080E94461519E115C0163111F0D0
:1053700015E211C082E30E94281584E00E942815DE
:10538000609121087091220880912308909124084F
:105390000E9446151FE187E30E94281586E00E94BF
:1053A000281581E00E94281583E00E94281586E0D8
:1053B0000E94281583E30E9428158AE30E9428157D
:1053C0008BE30E9428158DE30E94281587E00E9438
:1053D000281581E00E94281580E091E066E070E0E9
:1053E0000E945F158FEF0E942815101B80E0612F2F
:1053F00070E00E9477158CE291E00E946B261F916D
:105400000F910895EF92FF920F931F938091590887
:1054100090915A08892B59F4A8E0B1E0EDE1F1E050
:1054200082E101900D928150E1F760E0DCC0809153
:105430005808813031F0863121F0883111F08931FE
:10544000D9F5E0905508F090560800E010E088E0AB
:1054500091E06DE171E00E94D23EE61AF70A080B76
:10546000190BE0925108F0925208009353081093E0
:1054700054081E141F0410061106F4F080915808F9
:10548000813049F0863159F480915B088F5F8093B9
:105490005B08833018F00E94212803C086E10E9437
:1054A000FF28682FA8E0B1E0EDE1F1E082E1019092
:1054B0000D928150E1F701C060E0E0904D08F0905E
:1054C0004E0800914F0810915008D801C70101966D
:1054D000A11DB11D0297A105B10508F484C08091FA
:1054E000450890914608A0914708B091480820913E
:1054F000490830914A0840914B0850914C08009758
:10550000A105B10591F10197A109B1098093450861
:1055100090934608A0934708B09348082150304024
:10552000404050402093490830934A0840934B082C
:1055300050934C080894E108F10801091109E09220
:105540004D08F0924E0800934F08109350080097B2
:10555000A105B10509F047C088E10E94FF28682F26
:10556000882309F040C06CE03EC00894E108F108CF
:1055700001091109211531054105510509F1DA012A
:10558000C9010197A109B1098093490890934A087C
:10559000A0934B08B0934C08E0924D08F0924E084F
:1055A00000934F08109350080097A105B105D9F456
:1055B00089E10E94FF28682F8823A9F46DE013C0B9
:1055C000E0924D08F0924E0800934F081093500857
:1055D000E114F1040105110531F40E942128682F1E
:1055E000882309F46EE0862F1F910F91FF90EF90B2
:1055F0000895ACE1B0E0EFEFFAE20C942E628091F6
:105600005808882309F4E8C1873109F4E5C180917D
:10561000B0049091B10480519F4F0E94D5150E9413
:10562000D614182F8F3F09F4C5C00E94D614082F36
:10563000153341F4813009F0D6C10E94D61480930D
:105640005708EDCF113071F4843009F0CCC10E94BD
:10565000F51460932508709326088093270890938B
:105660002808DDCF133071F4843008F4BCC10E94E7
:10567000F5146093290870932A0880932B0890935F
:105680002C081FC0163371F4843008F4ACC10E949A
:10569000F51460932D0870932E0880932F08909333
:1056A00030080FC01630A1F4843008F49CC10E9469
:1056B000F514609331087093320880933308909307
:1056C0003408043009F4ABCF802F90E004976FC00A
:1056D000133309F04BC0843009F0A1CF0E94F514B8
:1056E0007B018C0160933D0870933E0880933F08D6
:1056F000909340088091390890913A08A0913B0816
:10570000B0913C080097A105B105B1F4C801B701FB
:105710002BE633E040E050E00E94A66128EE33E043
:1057200040E050E00E94E5612093390830933A0848
:1057300040933B0850933C0880913508909136087F
:10574000A0913708B09138080097A105B10509F07C
:1057500066CF16950795F794E794E0923508F09296
:105760003608009337081093380859CF1A3371F46C
:10577000843009F054CF0E94F5146093350870937B
:105780003608809337089093380849CF1B3371F45B
:10579000843009F044CF0E94F51460933908709367
:1057A0003A0880933B0890933C0839CF90E00E94E0
:1057B000191835CF8091B0049091B10404960E94DD
:1057C000D51580915808909157088130B9F49230DE
:1057D00009F004C10E94F51420914108309142085B
:1057E0004091430850914408621773078407950756
:1057F00009F0F4C083E00E94FF28F1C0953009F061
:10580000D9C00E94F514209141083091420840917E
:10581000430850914408621773078407950709F0FD
:10582000DDC087E1809358088091B0049091B10465
:1058300040960E94D5150E94F514AB01BC0140931F
:105840002D0550932E0560932F057093300588E049
:1058500090E00E9464638091250890912608A091B1
:105860002708B09128088093310590933205A093C2
:105870003305B09334058091290890912A08A091AE
:105880002B08B0912C088093350590933605A09392
:105890003705B09338058091310890913208A09176
:1058A0003308B09134088093E1099093E209A09302
:1058B000E309B093E4098091350890913608A091EE
:1058C0003708B09138088093450890934608A09314
:1058D0004708B09348088091390890913A08A09100
:1058E0003B08B0913C088093490890934A08A093E4
:1058F0004B08B0934C0880913D0890913E08A091D0
:105900003F08B091400880934D0890934E08A093B3
:105910004F08B09350088F5F9F4FAF4FBF4F21F498
:1059200010925A0810925908DE011196ECE9F4E041
:105930008CE101900D928150E1F760912D057091FD
:105940002E0580912F05909130050E946C1E0E94BB
:1059500014160E94C11A8C01A8950E94362081302D
:1059600019F40E94141609C0823039F40E94972756
:105970008823B1F40E94212813C00E94C11A801B01
:10598000910B8D54914040F38091E5098150823014
:1059900030F481E090E09093ED098093EC0980E091
:1059A000ACE9B4E0FE0131969CE101900D9291507A
:1059B000E1F715C0963091F40E94F514209141084A
:1059C0003091420840914308509144086217730790
:1059D0008407950719F407C080E001C08FE06C963A
:1059E000E6E00C944A620E942128F9CFAF92BF9260
:1059F000DF92EF92FF920F931F93DF93CF930F925B
:105A0000CDB7DEB7F82EE92E9C0159018EE2D82ED3
:105A10000E94D614982F882331F40894A108B10865
:105A2000F501108219C0807C803C11F085010AC00C
:105A30000E94D61411C099830E94D614F801819354
:105A40008F019981802F8A198917A8F3A90EB11C9B
:105A5000F501D1925F01DCCF8F2D9E2D0F90CF915C
:105A6000DF911F910F91FF90EF90DF90BF90AF906B
:105A70000895ACE4B0E0EFE3FDE20C942462809181
:105A8000B0049091B1040E94D515CE0101966CE04E
:105A900070E00E94111589819A810E94353E209103
:105AA000C6093091C7098217930709F06AC08D8132
:105AB0009E810E94353E6C01EE24FF243DE2A32E20
:105AC000B12CAC0EBD1E2DE0822E912C8C0E9D1E95
:105AD00014C0C5010E94F62C0E94E3148C010E94A0
:105AE000E3140130110531F4019721F4C401B5012B
:105AF0000E9402630894E11CF11CEC14FD0448F3BD
:105B00008F8198850E94353E3C01EE24FF249DE262
:105B1000492E512C4C0E5D1E31C0C2010E94F62C44
:105B20000E94E3148C010E94E3144C010E94F514BE
:105B30005B016C010E94E31401301105D1F421E0F6
:105B400082169104B1F48430910599F40E94F51401
:105B5000AB01BC014093C8095093C9096093CA09BD
:105B60007093CB09CE010D96960185010E945F319D
:105B700008C00E9419180894E11CF11CE614F704EF
:105B800060F280E0C45BDF4FE0E10C944062AF92D2
:105B9000BF92DF92EF92FF920F931F93CF93DF9309
:105BA000182F092F8091E1099091E209A091E30952
:105BB000B091E4098093A4049093A504A093A60453
:105BC000B093A70485E390E09093AD048093AC0478
:105BD00080E094E09093AF048093AE040E94C43DB3
:105BE0007093C7096093C6098AE290E00E94FA1593
:105BF0008091C6099091C7090E94351580E091E017
:105C00000E94351581E090E00E94351580E090E01B
:105C10000E94351580E090E00E94351580E090E00C
:105C20000E943515212F302FC901EC0140E1A42E2F
:105C3000B12C7E010E2D0C1BF701D080FEE2DF1689
:105C400031F0DD2021F00894E11CF11CF3CF802F0E
:105C50000E94281510E0CE01B8010E945F150F5F69
:105C60001F4FA00EB11EDD2019F0E7012196E1CFF4
:105C700080E00E94281581E090E00E94351581E0C7
:105C800090E00E943515C50101960E946B26DF91B8
:105C9000CF911F910F91FF90EF90DF90BF90AF9049
:105CA00008951F930E94D614182F11541295107F37
:105CB0000E94D61481548F70812B1F9108950F93E9
:105CC0001F93CF93DF93EC0100E0899190E00E9455
:105CD0006D62182F85958595859585958F5B0E94BA
:105CE00028151F70812F8F5B0E9428150F5F0031D0
:105CF00061F780E00E942815DF91CF911F910F91ED
:105D00000895ACE1B0E0E7E8FEE20C9424628091F3
:105D1000B0049091B1040E94D515CE0101966CE0BB
:105D200070E00E9411158B819C810E94353E9C0180
:105D30008F709070892B11F082E1EEC037FF5AC04E
:105D400089819A810E94353E2091C6093091C70908
:105D50008217930709F0DFC08F8198850E94353E36
:105D6000019711F080E1D8C00E94D614803211F062
:105D700081E1D2C08E01035F1F4FC801902E892E92
:105D80002DE1E22EF12CEC0EFD1E0E94512EF801A9
:105D900081938F01EE15FF05C1F71C8E0E94D6146A
:105DA0000E94E3148C010E94E3147C010E94F5140C
:105DB0005B016C010032110509F0ADC0F1E0EF1696
:105DC000F10409F0A8C00E94E3140E94E3140E94A9
:105DD000F514AB01BC014093C8095093C909609305
:105DE000CA097093CB09892D982D960185010E94CF
:105DF0005F3191C020703877232B09F08CC08091DF
:105E0000B2049091B304C29709F085C089819A8148
:105E10000E94353E4C018D819E810E94353E5C0181
:105E2000CC24DD249DE0692E712C6C0E7D1E8DE14D
:105E3000482E512C4C0E5D1E31C00E94D61480326B
:105E400009F069C083010E94512EF80181938F01EE
:105E5000E415F505C1F71C8E0E94D6140E94E314C8
:105E60007C010E94E3140197B1F4F0E2EF16F10413
:105E700051F4C30161ED79E00E94F962009759F491
:105E800000E015E84FC081E2E816F10421F48D85A9
:105E90008A3209F445C00894C11CD11CCA14DB0421
:105EA00060F239C086E090E00E94351580E090E015
:105EB0000E94351560912D0570912E0580912F055A
:105EC000909130050E9446158EE390E021C08DE34D
:105ED00090E00E94351581E00E94281581ED99E03F
:105EE0006FE070E00E945F1580E00E94281580E05E
:105EF00094E00E94351580E091E066E070E00E9439
:105F00005F1580E064E270E00E94771585E790E01D
:105F10000E946B2601C080E06C96E0E10C94406228
:105F200000E014E88AE290E00E94FA15C4010E94A1
:105F30003515C8010E94351580E090E00E943515A6
:105F400081E090E00E94351580E090E00E943515D8
:105F500080E090E00E94351580E20E942815CE0175
:105F60000D960E945F2EC7010E94351581E090E0DA
:105F70000E94351568E572E080E090E00E944615C9
:105F8000E0E2EE16F10409F0A2CF8CCF0F931F933D
:105F90008C018091310590913205A0913305B0912B
:105FA000340580959095A095B09520912D05309160
:105FB0002E0540912F0550913005822B932BA42B59
:105FC000B52B8093A4049093A504A093A604B0934A
:105FD000A70489E890E09093AD048093AC0490937B
:105FE000AF048093AE040E94C43D7093C7096093D0
:105FF000C6098AE290E00E94FA158091C609909144
:10600000C7090E94351580E191E00E94351581E0B5
:1060100090E00E94351580E090E00E94351580E008
:1060200090E00E94351580E090E00E94351580E2F6
:106030000E942815C8010E945F2E80E290E00E9415
:10604000351581E090E00E94351582E390E00E94D2
:106050006B261F910F910895E0EAF8E0848181306A
:10606000A1F480819181A281B3810097A105B1053E
:1060700061F00197A109B10980839183A283B38361
:106080000097A105B10509F41482B99689E0E83EAC
:10609000F80721F70895A9E2B0E0E1E5F0E30C94F8
:1060A0002C627C010CE718E06E010894C11CD11C25
:1060B000D601F80189E201900D928150E1F789A59E
:1060C000813059F4C601B7010E94F962009729F4A2
:1060D00029A13AA14BA15CA10AC0075D1F4F89E02D
:1060E000043C180729F720E030E040E050E0B90117
:1060F000CA01A996E8E00C944862CF93DF9380919F
:10610000CE09813001F5CCE5D8E0CE0168EC79E02C
:106110000E943F3E813009F4C3C0FE01019000207F
:10612000E9F73197EC1BFD0B709738F4CE016EE266
:1061300070E00E94EE62009711F084E001C082E0FE
:106140008093CE09A9C0823009F58CE598E00E94C1
:106150004B306093C8097093C9098093CA09909322
:10616000CB09611571058105910509F099C00E945F
:10617000C11A9093C5098093C4098CE598E00E94E8
:10618000C62F282F1092CD0983E053C0833079F5B4
:106190008091C8099091C909A091CA09B091CB0911
:1061A0000097A105B10509F07BC00E94C11A20919A
:1061B000C4093091C509821B930B885E934008F493
:1061C0006BC08091CD098F5F8093CD09833020F023
:1061D0002091F4072D5E61C00E94C11A9093C509F9
:1061E0008093C4098CE598E00E94C62F53C0843088
:1061F00019F58CE598E00E944B306093C8097093C4
:10620000C9098093CA099093CB096115710581056D
:10621000910509F045C00E94C11A9093C509809369
:10622000C4098CE598E00E94C72D282F1092CD0953
:1062300085E08093CE0931C0853071F58091C80921
:106240009091C909A091CA09B091CB090097A10505
:10625000B10531F50E94C11A2091C4093091C509D8
:10626000821B930B885E9340B8F08091CD098F5FBD
:106270008093CD09833020F02091F407295E0DC072
:106280000E94C11A9093C5098093C4098CE598E0D7
:106290000E94C72D282F01C020E080E090E003C0BD
:1062A00020E081E090E09093D0098093CF0901979E
:1062B00011F41092CE09822FDF91CF910895A0E0C2
:1062C000B0E0E5E6F1E30C942662EC016A017B01A3
:1062D0004801590100E010E089E2682E712C069D0A
:1062E000C001079D900D169D900D11248458974F65
:1062F000BE010E94F962009739F10F5F1F4F08300D
:10630000110569F72091CC09822F8F5F87708093E8
:10631000CC0930E089E290E0289F8001299F100D90
:10632000389F100D11240458174FC801BE010E9458
:106330000263F801C0A2D1A2E2A2F3A284A295A2B4
:10634000A6A2B7A281E080A7CDB7DEB7EEE00C949D
:106350004262A8E0B0E0EFEAF1E30C942A626D83B8
:106360007E838F83988719821A821B821C822981DF
:106370003A814B815C81F8EEAF2EE3E0BE2ECC2457
:10638000DD24EE24FF2400E010E00E94315B952F15
:10639000B901842F2896EAE00C944662A4E2B0E0AA
:1063A000E4EDF1E30C942C621091F4071093F507DF
:1063B00000E0B5E0EB2EF12CEC0EFD1E6E01089412
:1063C000C11CD11C1F5F1370E12FF0E0EE0FFF1F07
:1063D000EC5AFE4F65917491C7010E940263C70198
:1063E000B6010E943F3E813041F489819A81AB81A0
:1063F000BC810097A105B10519F01093F40703C003
:106400000F5F0430F9F6A496E8E00C944862AF926E
:10641000BF92CF92DF92EF92FF920F931F93609300
:10642000A4047093A5048093A6049093A7048BE71B
:1064300090E09093AD048093AC049093AF0480936C
:10644000AE048AE290E00E94FA1583E20E942815C9
:1064500080E067E270E00E947715F894E090020C0B
:10646000F090030C0091040C1091050C6091000C4D
:106470007091010C882777FD8095982F0E94A93193
:106480005B016C0178946093060870930708809311
:1064900008089093090880E89EE7AAEAB3E8E80EA6
:1064A000F91E0A1F1B1FC801B7010E944615C6012D
:1064B000B5010E94461580E390E00E946B261F9173
:1064C0000F91FF90EF90DF90CF90BF90AF90089525
:1064D0001F931091F609112309F480C01130A1F423
:1064E0008091F407E82FF0E0EE0FFF1FEC5AFE4F0B
:1064F000659174918CE598E00E9402631093CE0937
:1065000082E08093F6096AC0123089F58091CF0944
:106510009091D009019709F061C01092D0091092B2
:10652000CF096091C8097091C9098091CA099091F9
:10653000CB096093700770937107809372079093F3
:10654000730710921E080E940732182F882351F4F7
:1065500083E08093F6090E94C11A909317088093F4
:10656000160802C01092F6090E94CE3138C01330CE
:10657000A9F50E94C11A2091160830911708821BB4
:10658000930B20911808309119088217930730F166
:1065900080911E088F5F80931E08833040F0109317
:1065A0007D011091F507145E0E94950B18C0609153
:1065B00070077091710780917207909173070E9424
:1065C0000732182F882339F40E94C11A90931708B4
:1065D0008093160804C01092F60901C010E0812FC4
:1065E0001F9108958091E7098770823019F484EF34
:1065F00090E004C0833041F480EF90E00E942C18BA
:1066000080E00E942815089560912D0570912E0557
:1066100080912F05909130050E9446150895AF9204
:10662000BF92CF92DF92EF92FF920F931F938091D0
:10663000FA079091FB07A091FC07B091FD078093AA
:10664000A4049093A504A093A604B093A7048BE799
:1066500090E09093AD048093AC049093AF0480934A
:10666000AE048091F7099091F809892B19F405EE91
:1066700010E102C005E211E08AE290E00E94FA1502
:10668000802F0E942815812F0E94281560911A08DA
:1066900070911B0820E030E84FE0C9018623972362
:1066A000892B29F4415019F036952795F6CF842F80
:1066B0000E94281586EF0E9428156091FE077091B0
:1066C000FF0780910008909101080E944615609193
:1066D00002087091030880910408909105080E94B7
:1066E00046150E94F232609114087091150880E0FE
:1066F00090E00E94A9317B018C0160910E0870919D
:106700000F088091100890911108605871488545D4
:106710009C470E944615C801B7010E94461580E0BB
:1067200060E170E00E947715F894E090020CF09020
:10673000030C0091040C1091050C6091000C7091F9
:10674000010C882777FD8095982F0E94A9315B0165
:106750006C01789480E89EE7AAEAB3E8E80EF91E97
:106760000A1F1B1FC801B7010E944615C601B501CB
:106770000E94461580E390E00E946B261F910F91C6
:10678000FF90EF90DF90CF90BF90AF900895A7E675
:10679000B0E0EDECF3E30C9422628091B0049091B0
:1067A000B1040E94D515CE01819660E370E00E948D
:1067B000111599A1892F8770843009F01CC480912C
:1067C000F609882309F49AC7892F807C80930601F3
:1067D0009AA1803C21F0992311F0903158F082E089
:1067E00080937D011092CE091092F6090E94950BBC
:1067F0008BE185C79F5F909307016DA17EA18FA15B
:1068000098A50E94393E6093FE077093FF0780931E
:1068100000089093010869A57AA58BA59CA50E9404
:10682000393E6093020870930308809304089093A4
:106830000508FE01E05CFF4F90812FAD5EAD6DADB0
:106840007CADABADDAAC99ACFE01EC5BFF4FC08028
:10685000FE01ED5BFF4FB080FE01EE5BFF4FA080BD
:10686000FE01EF5BFF4F7080FE01E85BFF4F808110
:10687000FE01E95BFF4F3081FE01EA5BFF4F408183
:10688000FE01EB5BFF4FE081E82EE91A91E08E15E7
:1068900008F090E0832F821B21E0381708F020E0F9
:1068A000F82EF91A91E08F1508F090E0292B842F2B
:1068B000851B31E0481708F030E0082F021B91E0FB
:1068C000801708F090E0392B8E2F861B21E0E81707
:1068D00008F020E0182F131B91E0811708F090E0DA
:1068E000292B8C2D871B31E0C81608F030E0B82F1B
:1068F000B21B91E08B1708F090E0392B8B2D8A1B8F
:1069000021E0B81608F020E0A82FA31B91E08A1719
:1069100008F090E0292B8A2D8D1991E0A81608F037
:1069200090E0F82FF21B21E08F1708F020E0922B67
:10693000E72DE919E91B9701A8016B2F7A2F8F2FFB
:106940009E2F52F52E2D2F5F81E02E1508F080E04E
:10695000382F3F0D81E03F1508F080E0482F400FB1
:1069600081E0401708F080E0582F510F81E0511767
:1069700008F080E0682F6B0F81E06B1708F080E073
:10698000782F7A0F81E07A1708F080E08F0F91E07E
:106990008F1708F090E09E0F01E00E94AC5A622E23
:1069A000532E442E352E262E62967FAF6297639625
:1069B0008FAF639764969FAF6497FE01E45BFF4FD0
:1069C000C080FE01E55BFF4FB080FE01E65BFF4F3C
:1069D000A080FE01E75BFF4F7080FE01E05BFF4F90
:1069E0000081FE01E15BFF4FF080FE01E25BFF4FA3
:1069F0009080FE01E35BFF4F808080910A089091B8
:106A00000B08A0910C08B0910D0880589148A5453D
:106A1000BC47182F8D8B9E8BAF8BB88F609112085F
:106A20007091130880E090E00E94A931698B7A8B05
:106A30008B8B9C8B872F3B89492F5E897F89E88DC3
:106A4000D02ED61A91E00D1508F090E02F2D281BBE
:106A5000822F21E0F81608F020E0E82EE91A91E0F4
:106A60008E1508F090E0292B892D831B31E09816B4
:106A700008F030E0F82EF21A91E08F1508F090E05F
:106A8000392B882D841B21E0881608F020E0082F80
:106A9000031B91E0801708F090E0292B3C2D311B5F
:106AA000132F91E0C31608F090E0B12FB21B81E0E4
:106AB0001B1708F080E0982B8B2D851B21E0B81662
:106AC00008F020E0A82FA91B91E08A1708F090E0B9
:106AD000292B8A2D871B91E0A81608F090E0F82F4B
:106AE000F21B21E08F1708F020E0922B7E1AE72D91
:106AF000E91B2D2D3E2D4F2D502F6B2F7A2F8F2FD1
:106B00009E2F52F52D2D2F5F81E02D1508F080E08E
:106B1000382F3E0D81E03E1508F080E0482F4F0DE4
:106B200081E04F1508F080E0582F500F81E050179A
:106B300008F080E0682F6B0F81E06B1708F080E0B1
:106B4000782F7A0F81E07A1708F080E08F0F91E0BC
:106B50008F1708F090E09E0F01E00E94AC5AA32F1F
:106B6000B42F152F062FF72ED82EC22EC60CF1E00B
:106B7000C21608F0F0E03A2F350DE1E03A1708F0C0
:106B8000E0E0EF2EE30E21E0E31608F020E0E22B38
:106B90004B2F440D31E04B1708F030E0AE2FA40F1F
:106BA00021E0A41708F020E0322B512F530D41E0D3
:106BB000511708F040E0F32FF50F21E0F51708F02A
:106BC00020E0422B602F620D31E0601708F030E0CA
:106BD000E42FE60F21E0E61708F020E0322B629662
:106BE0007FAD62977F0D41E07F1508F040E0532FA5
:106BF000570F21E0571708F020E0422B63968FAD26
:106C000063978D0D21E08D1508F020E0480F31E0ED
:106C1000481708F030E0232B64968FAD6497980FE7
:106C2000290FC98AEA8AAB8BFC8BED8B5E8B4F8B6D
:106C3000288F4D885E886F88788C89899A89AB897E
:106C4000BC894C015D01CC24DD2476019C01A501A9
:106C500060E070E080E090E002E00E942D5A122F88
:106C6000232E65964FAF659766965FAF66976796DA
:106C70006FAF679768967FAF689769968FAF699790
:106C80006A969FAF6A9705E00E942D5AA32FB42FF2
:106C9000052F6B966FAF6B976C967FAF6C976D9669
:106CA0008FAF6D976E969FAF6E97322E311AF1E0CF
:106CB000231508F0F0E03A2F3219E1E0A31708F0AD
:106CC000E0E0132F1F1B21E0311708F020E0E22B3A
:106CD0004B2F65969FAD6597491B31E0B41708F0BF
:106CE00030E0B42FBE1B21E04B1708F020E0322B20
:106CF000502F6696AFAD66975A1B41E0051708F016
:106D000040E0052F031B21E0501708F020E0422B44
:106D10006B966FAD6B976796EFAD67976E1B31E023
:106D20006B96FFAD6B97F61708F030E0962F941B2B
:106D300021E0691708F020E0322B6C967FAD6C974C
:106D400068962FAD6897721B41E06C968FAD6C977B
:106D5000871708F040E0A72FA31B21E07A1708F05F
:106D600020E0422B6D968FAD6D976996EFAD6997D8
:106D70008E1B21E06D96FFAD6D97F81708F020E0AF
:106D8000E82FE41B31E08E1708F030E0232B6E96DD
:106D9000FFAD6E976A963FAD6A97F31BF21B232CEB
:106DA000280C31E0231408F030E0812F890D41E0F8
:106DB000811708F040E0380F51E0381708F050E034
:106DC000452B8B2F8A0D51E08B1708F050E0480FB0
:106DD00061E0481708F060E0562B202F2B0D81E072
:106DE000201708F080E0520F61E0521708F060E0D1
:106DF000682B690F71E0691708F070E07A0F81E085
:106E00007A1708F080E08E0F91E08E1708F090E07E
:106E1000222D9F0F03E00E942D5A298F3A8F4B8F0E
:106E20005C8F6D8F7E8F8F8F98A3ED8CFE8C0F8D76
:106E300018A180911B0190911C01892BC9F48091AC
:106E40001F0890912008009799F0A301920177FE06
:106E500007C022273327A9012419350946095709F4
:106E6000A0E0B0E082179307A407B5070CF446C46E
:106E70008701F8948091020C9091030CA091040C6E
:106E8000B091050C840D951DA61DB71D8093020CB5
:106E90009093030CA093040CB093050C8091000C0C
:106EA0009091010C8E0D9F1D9093010C8093000C0E
:106EB0008091000C9091010C97FF2AC08091020CE8
:106EC0009091030CA091040CB091050C18161906B2
:106ED0001A061B06ECF48091020C9091030CA09111
:106EE000040CB091050C0197A109B1098093020C23
:106EF0009093030CA093040CB093050C8091000CAC
:106F00009091010C88519C4F9093010C8093000C40
:106F10008091020C9091030CA091040CB091050C8F
:106F200080930E0890930F08A0931008B093110857
:106F30008091000C9091010C909315088093140897
:106F4000789477FE0AC0101611063CF40894411C90
:106F5000511C611C711C085E1340D301C20180509A
:106F60009048AF4FBF4F80509040A140B04038F0A4
:106F70008FEF9FE79093F7078093F60704C0509236
:106F8000F7074092F6071093F9070093F8078091EE
:106F9000FF09882361F1C301B20128EE33E040E02C
:106FA00050E00E94A6619B01AC01C801AA2797FD91
:106FB000A095BA2F820F931FA41FB51FB7FD04C061
:106FC000B801620F731F0AC0C301B20128E13CEF90
:106FD0004FEF5FEF0E94A661601B710B7093FE097B
:106FE0006093FD096D54714014F081E001C082E0AE
:106FF0008093FF097DC3833009F0D6C0292F287301
:107000008091F7099091F809019701F550900601D8
:10701000522A40900701E0900E08F0900F0800916E
:1070200010081091110880E89EE7AAEAB3E8E80E7C
:10703000F91E0A1F1B1F609114087091150880E04B
:1070400090E00E94A9313B014C010BC040EC542E52
:10705000522A662477244301EE24FF24870130E17D
:10706000432EA0900A08B0900B08C0900C08D09056
:107070000D0820901208309013088AE290E00E94D8
:10708000FA15852D84600E942815842D0E942815EC
:107090008BA10E94281586EF0E94281560E070E001
:1070A00080E090E00E94461560E070E080E090E0B3
:1070B0000E9446150E94F232C801B7010E9446158F
:1070C000C401B3010E9446158091F7099091F80917
:1070D000019799F4CE0181968C01085D1F4F20E342
:1070E000E22EF12CE80EF91ED8018D918D010E943F
:1070F00028150E151F05C1F70CC060E070E080E098
:1071000090E00E94461560E070E080E090E00E9410
:10711000461580E89EE7AAEAB3E8A80EB91ECA1E83
:10712000DB1EC601B5010E944615B10180E090E06A
:107130000E94A9310E9446158091F7099091F809A3
:10714000019739F0AA24BB246501EE24FF248701AE
:107150001EC0F894E090020CF090030C0091040C17
:107160001091050C80E89EE7AAEAB3E8E80EF91E44
:107170000A1F1B1F6091000C7091010C882777FD7E
:107180008095982F0E94A9315B016C017894C80109
:10719000B7010E944615C601B5010E94461580E35D
:1071A00090E00E946B26ABC2853009F0A7C28091A7
:1071B000E7098770813009F0A1C2892F807C809314
:1071C00006019AA1803C09F499C2992309F496C258
:1071D000903109F493C29F5F909307016DA17EA146
:1071E0008FA198A50E94393E6093FE077093FF0718
:1071F000809300089093010869A57AA58BA59CA5AA
:107200000E94393E6093020870930308809304083B
:1072100090930508FE01E05BFF4FD080FE01E15B2B
:10722000FF4FC080FE01E25BFF4FA080FE01E35BE9
:10723000FF4F10813D2DD9822C2DCA829A2DAB8211
:10724000812F1C83FE01E45BFF4FD080FE01E55BD4
:10725000FF4FC080FE01E65BFF4FA080FE01E75BB1
:10726000FF4F1081DD82CE82AF821887032FF22E6E
:10727000E92EB82E832F822B892B8B298D298C29DF
:107280008A29812B09F43AC2F8948091020C9091DA
:10729000030CA091040CB091050C80589148A545B1
:1072A000BC478D839E83AF83B8876091000C70913B
:1072B000010C882777FD8095982F0E94A93169835A
:1072C0007A838B839C83789489812A813B814C814A
:1072D0005D81AE81BF819884F02FF81B91E00F177C
:1072E00008F090E08F2D821B21E0F81608F020E0D6
:1072F000E82FE91B91E08E1708F090E0292B8E2DE6
:10730000831B31E0E81608F030E0782F721B91E023
:10731000871708F090E0392B8B2D841B21E0B816DD
:1073200008F020E0682F631B91E0861708F090E0DA
:10733000292B8D2D851B31E0D81608F030E0582F11
:10734000521B91E0851708F090E0392B8C2D8A1B99
:1073500021E0C81608F020E0482F431B91E0841775
:1073600008F090E0292B8A2D8B1B91E0A81608F0DD
:1073700090E0382F321B21E0831708F020E0922B99
:107380001919191BF983EA837B836C835D834E8310
:107390003F8318874D805E806F80788489819A81D1
:1073A000AB81BC814C015D01CC24DD2476019C01C4
:1073B000A50160E070E080E090E002E00E942D5ABC
:1073C000122F232E6F964FAF6F97A0965FAFA097A7
:1073D000A1966FAFA197A2967FAFA297A3968FAF0A
:1073E000A397A4969FAFA49705E00E942D5AA32FC0
:1073F000B42F052FA5966FAFA597A6967FAFA6973A
:10740000A7968FAFA797A8969FAFA897322E311A4D
:10741000F1E0231508F0F0E03A2F3219E1E0A3176C
:1074200008F0E0E0132F1F1B21E0311708F020E0E7
:10743000E22B4B2F6F969FAD6F97491B31E0B4172E
:1074400008F030E0B42FBE1B21E04B1708F020E01D
:10745000322B502FA096AFADA0975A1B41E00517D5
:1074600008F040E0052F031B21E0501708F020E052
:10747000422BA5966FADA597A196EFADA1976E1B78
:1074800031E0A596FFADA597F61708F030E0962FEE
:10749000941B21E0691708F020E0322BA6967FADFF
:1074A000A697A2962FADA297721B41E0A6968FAD2C
:1074B000A697871708F040E0A72FA31B21E07A17B3
:1074C00008F020E0422BA7968FADA797A396EFADCB
:1074D000A3978E1B21E0A796FFADA797F81708F09A
:1074E00020E0E82FE41B31E08E1708F030E0232B7A
:1074F000A896FFADA897A4963FADA497F31BF21BE7
:10750000232C280C31E0231408F030E0812F890D62
:1075100041E0811708F040E0380F51E0381708F0DB
:1075200050E0452B8B2F8A0D51E08B1708F050E06F
:10753000480F61E0481708F060E0562B202F2B0D14
:1075400081E0201708F080E0520F61E0521708F048
:1075500060E0682B690F71E0691708F070E07A0F3E
:1075600081E07A1708F080E08E0F91E08E1708F026
:1075700090E0222D9F0F03E00E942D5A29873A8721
:107580004B875C876D877E878F87988BED84FE8421
:107590000F85188980911B0190911C01892BC9F4DA
:1075A00080911F0890912008009799F0A301920103
:1075B00077FE07C022273327A90124193509460978
:1075C0005709A0E0B0E082179307A407B5070CF4B1
:1075D00095C09701F8948091020C9091030CA091B2
:1075E000040CB091050C840D951DA61DB71D80934C
:1075F000020C9093030CA093040CB093050C8091A3
:10760000000C9091010C8E0D9F1D9093010C8093A6
:10761000000C8091000C9091010C97FF2AC0809182
:10762000020C9091030CA091040CB091050C18165B
:1076300019061A061B06ECF48091020C9091030CBB
:10764000A091040CB091050C0197A109B109809398
:10765000020C9093030CA093040CB093050C809142
:10766000000C9091010C88519C4F9093010C8093D9
:10767000000C8091020C9091030CA091040CB0912D
:10768000050C80930E0890930F08A0931008B093F8
:1076900011088091000C9091010C90931508809333
:1076A0001408789477FE0AC0121613063CF4089466
:1076B000411C511C611C711C285E3340D301C20166
:1076C00080509048AF4FBF4F80509040A140B04095
:1076D00038F08FEF9FE79093F7078093F60704C089
:1076E0005092F7074092F6073093F9072093F80776
:1076F00081E090E09093090C8093080C80E0C959D8
:10770000DF4FE2E10C943E628091F7099091F80915
:10771000892B11F480E008958AE290E00E94FA1526
:10772000F8946091020C7091030C8091040C90917C
:10773000050C78946058714885459C470E94461511
:1077400084E090E00E946B260895DB01982F9295CB
:107750009F702CE531E0F901E90FF11DE491EC9304
:107760008F70280F311DF901849111968C93119718
:1077700012961C921297CB010895DB01292F2295B6
:107780002F704CE551E0FA01E20FF11DE491EC930A
:107790009F70FA01E90FF11DE4911196EC93119796
:1077A000982F92959F70FA01E90FF11DE4911296BE
:1077B000EC9312978F70480F511DFA018491139624
:1077C0008C93139714961C921497CB010895DA01A9
:1077D000292F22952F704CE551E0FA01E20FF11D9F
:1077E000E491EC939F70FA01E90FF11DE491119679
:1077F000EC931197982F92959F70FA01E90FF11D64
:10780000E4911296EC9312978F70FA01E80FF11D34
:10781000E4911396EC931397872F82958F70FA015A
:10782000E80FF11DE4911496EC9314977F70FA0120
:10783000E70FF11DE4911596EC931597862F82952D
:107840008F70FA01E80FF11DE4911696EC931697EC
:107850006F70460F511DFA01849117968C931797FC
:1078600018961C921897CD010895282FDB0164E625
:107870000E94C561392F822F0E94C561805DFD0184
:107880008193832F6AE00E94C561805D11968C937D
:107890001197832F0E94C561905D91831282CD0163
:1078A0000895A0E0B0E0E7E5FCE30C942D62482FDA
:1078B000F92EE62ED72E862F972F9C01E901E0E1C5
:1078C000F7E200E010E0842F9F2DBF010E94D161FC
:1078D000262F842F9F2DBF010E94D161482FF92EA2
:1078E000205D2993CF016AE070E00E94D161FB0125
:1078F0000F5F1F4F0430110531F7405D4883198237
:107900008E2D9D2DCDB7DEB7E7E00C944962A0E047
:10791000B0E0EDE8FCE30C942562062F772E4C01D5
:10792000642E552E842F952F9C01E901C12C8AECE1
:10793000D82E8AE9E82E8BE3F82EAA24BB24602FE8
:10794000772DC401A70196010E94E561122F602FD7
:10795000772DC401A70196010E94E561062F772EBD
:107960004C01105D1993C701B6012AE030E040E0F8
:1079700050E00E94E561C901DA016C017D010894C3
:10798000A11CB11C89E0A816B104C9F6005D0883EA
:107990001982862D952DCDB7DEB7EFE00C944162AC
:1079A000EF92FF920F931F938B019C01F42EE52E13
:1079B00097FD04C0842F952FFC010CC030952095B5
:1079C000109501951F4F2F4F3F4F842F952FFC018E
:1079D0008DE28193C901B801AF010E94873C8F2DD0
:1079E0009E2D1F910F91FF90EF9008951F93CF93BD
:1079F000DF93EC0120E030E040E050E01881812F7F
:107A000080538A30C8F4CA01B9012AE030E040E06E
:107A100050E00E94A6619B01AC01812F992787FD50
:107A20009095C097AA2797FDA095BA2F280F391FC8
:107A30004A1F5B1F2196E2CF203080E0380781E0AB
:107A4000480780E0580720F02FEF3FEF40E050E07C
:107A5000C901DF91CF911F910895982F81548630ED
:107A600010F487E307C0892F8156863010F487E52C
:107A700001C080E3981B892F0895FF920F931F93F5
:107A80008C01FC0180810E942D3DF82EF29490EF34
:107A9000F922F80181810E942D3D8F708F291F915D
:107AA0000F91FF900895EF92FF920F931F938C0117
:107AB000FC0180810E942D3DF82EF29430EFF322DC
:107AC000F80181810E942D3D8F70F82AF801828192
:107AD0000E942D3DE82EE29420EFE222F8018381FE
:107AE0000E942D3D8F708E299F2D1F910F91FF9029
:107AF000EF900895CF92DF92EF92FF920F931F9332
:107B00008C01FC0180810E942D3DC82EC29470EF33
:107B1000C722F80181810E942D3D8F70C82AF8018B
:107B200082810E942D3DD82ED29460EFD622F8019A
:107B300083810E942D3D8F70D82AF80184810E9494
:107B40002D3DF82EF29450EFF522F80185810E9428
:107B50002D3D8F70F82AF80186810E942D3DE82E78
:107B6000E29440EFE422F80187810E942D3D8F705E
:107B70008E29682F7F2D8D2D9C2D1F910F91FF90A9
:107B8000EF90DF90CF900895EF92FF920F931F93A5
:107B900080917E0190917F01A0918001B09181013F
:107BA0007C018D012BE0EE0CFF1C001F111F2A959C
:107BB000D1F7E826F9260A271B27809182019091A8
:107BC0008301A0918401B091850180937E019093FF
:107BD0007F01A0938001B0938101809186019091F3
:107BE0008701A0918801B0918901809382019093CF
:107BF0008301A0938401B093850180918A019091C3
:107C00008B01A0918C01B0918D018093860190939E
:107C10008701A0938801B09389019C01AD01F3E134
:107C20005695479537952795FA95D1F728273927FF
:107C30004A275B272E253F2540275127EF2CF02E82
:107C4000012F11272E253F254027512720938A01F8
:107C500030938B0140938C0150938D01B901CA017F
:107C60001F910F91FF90EF900895282F892F922F49
:107C70000895362F272F692F782FC9010895A0E284
:107C8000B0E0E5E4FEE30C9428629C015B018E0108
:107C90000F5F1F4FC801B9010E940263CC24DD248D
:107CA0007601980140E1842E912C8C0E9D1EF801E6
:107CB00080818E3291F41082C9010E94F63CA0E0CE
:107CC000B0E08C299D29AE29BF29CC24D82EE92EDD
:107CD000FA2E98012F5F3F4F2BC08823E9F4CE0185
:107CE00001960817190731F4F501108211821282EA
:107CF000138210C0F8011082C9010E94F63CA0E076
:107D0000B0E08C299D29AE29BF29F501808391839C
:107D1000A283B38381E013C0992787FD9095C09714
:107D20000A9730F0F501108211821282138206C088
:107D30000815190519F00F5F1F4FB9CF80E0A09605
:107D4000ECE00C944462CF92DF92EF92FF920F939B
:107D50001F936B01E82E8A01892FBA010E94353CDE
:107D60005EE2F52EF801F382B8016C5F7F4F8E2D35
:107D70000E94353CF801F782B801685F7F4F8D2D76
:107D80000E94353CF801F386B801645F7F4F8C2D6B
:107D90000E94353CC8011F910F91FF90EF90DF903A
:107DA000CF900895CF92DF92EF92FF920F931F939F
:107DB0006B010E94A81D7B018C01C6010E94A81DB9
:107DC0009B01AC012E193F09400B510BB901CA01AF
:107DD0001F910F91FF90EF90DF90CF900895A4E056
:107DE000B0E0E5EFFEE30C943062162F072F0E94FF
:107DF000A81D20917701309178014091790150912F
:107E00007A01260F371F481F591F29833A834B8356
:107E10005C83CE0101960E94001EAC01009711F414
:107E200080E00BC0812F902F9C01D901FA0182E1E3
:107E300001900D928150E1F781E02496E4E00C94EA
:107E40004C62A4E0B0E0E7E2FFE30C942C62D62E93
:107E5000C72E79018A010E94A81D6E197F09800B27
:107E6000910B69837A838B839C83CE0101960E9458
:107E7000001EAC01009711F480E00BC08D2D9C2DED
:107E80009C01D901FA0182E101900D928150E1F744
:107E900081E02496E8E00C944862EF92FF920F9301
:107EA0001F93E82EF62E8A01FA940E948B1BF8018C
:107EB0008083813131F48E2D8F5FF81660F480E07D
:107EC0000AC0823111F08E2D06C0EE2011F48F2DE4
:107ED00002C08E2D81501F910F91FF90EF90089559
:107EE000A0E0B0E0E6E7FFE30C942362C82E362E54
:107EF0007A01B22EE8010E94291AEB2DFF27E7FD37
:107F0000F095EE0DFF1D1082F7019081892F8053AF
:107F10008A3010F4182F08C0892F8154863010F051
:107F200010E002C0192F1753A8951B9BFDCF81E0CD
:107F30000E94DC19219711F08AE001C080E1012F35
:107F4000112707FD1095DC2CC0E0D0E04B2C552408
:107F500047FC5094882E992487FC9094340108940F
:107F6000610871085701AC0EBD1E8D2D632D0E9456
:107F7000F0190A30110518F4802F805D02C0802F9F
:107F8000895C0E94C0190E94D4190E948B1B813108
:107F900041F40F5F1F4F081519054CF000E010E089
:107FA00006C0823179F40150104017FD83010A3078
:107FB000110518F4802F805D02C0802F895CF501C7
:107FC0008083D0CF833151F52196D394F701EC0F04
:107FD000FD1F8081992787FD90950E945962892B0A
:107FE00011F42196D394C415D5051CF0DC2CC0E007
:107FF000D0E0F701EC0FFD1FE0818E2F80538A3017
:1080000040F08E2F8154863010F080E002C08E2F19
:108010008753082F112707FD1095A4CF843119F439
:1080200001E010E005C0893109F09CCF00E010E0CC
:1080300080E00E94DC19C801CDB7DEB7E1E10C9405
:108040003F628091140C8130C1F580910E0C9091AB
:108050000F0CA091100CB091110C0196A11DB11D37
:1080600080930E0C90930F0CA093100CB093110CF6
:1080700080910E0C90910F0CA091100CB091110CEE
:1080800080930E0890930F08A0931008B0931108E6
:108090008093020C9093030CA093040CB093050CF6
:1080A000109215081092140881E090E09093090C4A
:1080B0008093080C1092140C3EC08091120C8230F8
:1080C00099F08091020C9091030CA091040CB09156
:1080D000050C0196A11DB11D8093020C9093030C19
:1080E000A093040CB093050C8091E709877082304F
:1080F00031F52091E8093091E90921153105D9F0D0
:1081000080910C0C90910D0C019690930D0C809326
:108110000C0C80910C0C90910D0C8217930778F049
:1081200089E080937D0180917C01843041F083E07F
:1081300080937C0104C010920D0C10920C0C809165
:108140007C018130C1F48091EA099091EB09892B7F
:1081500091F080910A0C90910B0C019790930B0C6D
:1081600080930A0C80910A0C90910B0C892B19F4C6
:1081700082E080937C0181E090E09093070C8093F3
:10818000060C08951F920F920FB60F9211242F9391
:108190003F934F935F936F937F938F939F93AF938F
:1081A000BF93EF93FF9382E083BD1092B2001CBA9D
:1081B0001DBA88EC80937B018091140C8230C1F44D
:1081C0001092010C1092000C1092150810921408D5
:1081D00081E090E09093090C8093080C10920D0CB4
:1081E00010920C0C1092140C9093070C8093060CB8
:1081F0008091140C813091F48091E709877083306D
:1082000039F484E690E09093010C8093000C04C054
:108210001092010C1092000C0E9421408AE0809381
:10822000130CFF91EF91BF91AF919F918F917F912F
:108230006F915F914F913F912F910F900FBE0F90D3
:108240001F9018951F920F920FB60F9211240F9046
:108250000FBE0F901F9018951F920F920FB60F929E
:1082600011240F900FBE0F901F9018951F920F9220
:108270000FB60F9211242F933F934F935F936F93F9
:108280007F938F939F93AF93BF93EF93FF938091CF
:10829000000C9091010C01969093010C8093000CBE
:1082A0008091140C8230C9F41092010C1092000CD1
:1082B000109215081092140881E090E09093090C38
:1082C0008093080C10920D0C10920C0C1092140C50
:1082D0009093070C8093060C0DC08091000C909138
:1082E000010C885E9340BCF01092010C1092000CBF
:1082F0000E9421408091130C882331F08091130C4F
:1083000081508093130C07C080917D01873019F450
:1083100086E080937D01FF91EF91BF91AF919F9196
:108320008F917F916F915F914F913F912F910F901E
:108330000FBE0F901F9018951F920F920FB60F92BD
:1083400011248F939F938091BC029091BD0201965E
:108350009093BD028093BC0280917B01882359F0E9
:1083600080917B01815080937B0180917B018823E8
:1083700011F481E08DBB9F918F910F900FBE0F90F4
:108380001F9018951F920F920FB60F9211248F9382
:108390009F93EF93FF938091C0009091C6008C71E2
:1083A00079F480910804E82FF0E0E95FFC4F9083B6
:1083B0008F5F80930804809109048F5F8093090484
:1083C000FF91EF919F918F910F900FBE0F901F9093
:1083D00018951F920F920FB60F9211242F938F931F
:1083E0009F93EF93FF93209104032223B9F0909180
:1083F0000303E92FF0E0ED53FD4F80818093C60029
:108400009F5F90930303822F8150809304038823FE
:1084100029F48091C1008F7D8093C100FF91EF917D
:108420009F918F912F910F900FBE0F901F901895D5
:108430001F920F920FB60F9211248F938091040315
:10844000882349F48091C1008F7B8093C1001092F2
:108450000603109205038F910F900FBE0F901F908F
:108460001895CF93DF93EC0163E37BE044E050E0A9
:108470000E949962892B11F481E017C0CE016FE24E
:108480007BE043E050E00E949962892B11F482E086
:108490000CC0CE0168E27BE046E050E00E949962A9
:1084A000892B11F483E001C080E0DF91CF91089522
:1084B000CF93DF93019719F0C0E0D0E005C083E5CA
:1084C0009DE00E942C18EC0187E39DE00E942C188F
:1084D0009E01280F391FC901DF91CF910895A0E0B7
:1084E000B0E0E5E7F2E40C9424623B01E82FFF27BB
:1084F000E7FDF095EE0FFF1FED53F84F45905490B8
:1085000086EF9DE00E942C184C01C2010E942C189D
:10851000EC0188ED9DE00E942C185C01C2010E94D4
:108520002C186C018AEB9DE00E942C187C01C20182
:108530000E942C188C0186EA9DE00E942C18C80D20
:10854000D91DCA0DDB1DCC0DDD1DCE0DDF1DC00FED
:10855000D11FC80FD91F81E068167104A9F486E9FC
:108560009DE00E942C187C01C2010E942C188C01F5
:108570008BE79DE00E942C189701200F311F2C0FD4
:108580003D1F280F391F07C086E79DE00E942C1869
:108590009C012C0F3D1FC901CDB7DEB7E0E10C9463
:1085A0004062EF92FF920F931F93182F86E390E0A3
:1085B0000E94FA158EED91E00E942C187C01E12FAB
:1085C000FF27E7FDF095EE0FFF1FE35CF74F859166
:1085D00094910E942C188C018CE09EE00E942C1833
:1085E0000E0D1F1D080F191FC8011F910F91FF903D
:1085F000EF900895A0E0B0E0E0E0F3E40C942A628C
:10860000082F86E390E00E94FA158EED91E00E941B
:108610002C185C01C02FDD27C7FDD095CC0FDD1FC6
:10862000FE01E35CF74F859194910E942C188C0118
:1086300088E49EE00E942C186C01FE01ED53F84F77
:10864000859194910E942C187C018AE39EE00E94FF
:108650002C180A0D1B1D0C0D1D1D0E0D1F1D080FC6
:10866000191FC801CDB7DEB7EAE00C944662AF929D
:10867000BF92CF92DF92EF92FF920F931F938C01E4
:10868000F62EE72E89ED9CE00E942C185C01C801B3
:108690000E942C188C018FEC9CE00E942C186C011D
:1086A000EF2DFE2DDF010D900020E9F71197AE1B95
:1086B000BF0B8F2D9E2DBD010E945F157C0184ECA8
:1086C0009CE00E942C180A0D1B1D0C0D1D1D0E0D8B
:1086D0001F1D080F191FC8011F910F91FF90EF90E8
:1086E000DF90CF90BF90AF900895A4E0B0E0EBE7AB
:1086F000F3E40C943262BE016F5F7F4F0E94353C01
:10870000CE01029662E070E00E945F152496E2E0DE
:108710000C944E62A8E0B0E0E0E9F3E40C94266229
:108720007C01FC0180819181BE016F5F7F4F0E94BF
:10873000513CCE01029664E070E00E945F153C015E
:108740008FE20E942815F70182810E9475438C01F7
:108750008FE20E942815F70183810E9475434C0126
:1087600080E20E942815F70184810E9475435C0114
:108770008AE30E942815F70185810E9475436C01E8
:108780008AE30E942815F70186810E947543080D2F
:10879000191D0B5F1F4F0A0D1B1D0C0D1D1D080F12
:1087A000191F060D171DC8012896EEE00C944262B1
:1087B000A8E0B0E0EEEDF3E40C9422626C0180E3FB
:1087C0009DE00E942C189E838D83F601808191810B
:1087D0000E942C188C0182E19DE00E942C18988741
:1087E0008F83F601828193810E942C181C0189E0FD
:1087F0009DE00E942C182C01F60184817E010894D2
:10880000E11CF11CB7010E94353CF70101900020EA
:10881000E9F73197EE19FF09BF010E945F153C018E
:108820008BEF9CE00E942C184C01F6018581B7016A
:108830000E94353CF70101900020E9F73197EE19CD
:10884000FF09BF010E945F155C0181EF9CE00E945F
:108850002C187C01F60186819781FC01DF010D90C7
:108860000020E9F71197AE1BBF0BBD010E945F15F9
:108870002D813E81020F131FEF81F8850E0F1F1F00
:10888000020D131D040D151D060D171D080D191DD4
:108890000A0D1B1D0E0D1F1D080F191FC80128965C
:1088A000E2E10C943E62A8E2B0E0E9E5F4E40C9465
:1088B0002E62082F112707FD1095000F111FF801D8
:1088C000E75DFB4F85919491F801E45BFE4F459184
:1088D000549139E0E32EF12CEC0EFD1EB7010E94FD
:1088E000B61BF801EF5DFB4F859194919A838983C4
:1088F000F801E750FC4F859194919C838B8381E232
:108900008D838FE18E83F886EF82CE0101960E94DF
:10891000D843A896E6E00C944A62A8E1B0E0E3E907
:10892000F4E40C942E62E82EFF24E7FCF094870117
:10893000000F111FF801ED56FC4F8591949101C075
:10894000A895F999FDCF0E9436639B01AC012F3F9A
:108950008FEF38078FEF48078FEF580759F4F7016B
:10896000EE0FFF1FEE0FFF1FE356FC4F25913591D1
:1089700045915491F801ED51FC4F859194919A8362
:108980008983F801E757FC4F859194919C838B83F1
:1089900082E18D838FE08E83CA01B901AE01475F0A
:1089A0005F4F0E94A33E98878F83CE0101960E945D
:1089B000D8436896E6E00C944A62A0E0B0E0E3EEAB
:1089C000F4E40C942A625C0180E00E94FA426C019B
:1089D00080E00E948D44EC0181E00E948D447C0186
:1089E00082E00E948D448C0183E00E948D44CC0D76
:1089F000DD1DCE0DDF1DC00FD11FC80FD91F81E0B7
:108A0000A816B10419F48DE093E002C085E493E068
:108A10000E942C18C80FD91F81E090E00E94584294
:108A20006091680570916905C80FD91F88E1AE0192
:108A30000E94AA22CDB7DEB7EAE00C944662AAE90A
:108A4000B0E0E5E2F5E40C9422629C01880F991FE6
:108A5000BC01F3E0660F771FFA95E1F7680F791F05
:108A60006E5B7A4F7093690560936805F901E2596E
:108A7000F84FE081E13009F070C6232B29F0EAE6D7
:108A80008E2EE6E09E2E04C07AE6872E75E0972EA5
:108A9000C4016AE879E00E94A762FC01108263ECDD
:108AA000E62E67E0F62E00E0F70165917491C401AF
:108AB00046E050E00E949962892B09F455C00F5F8F
:108AC00022E030E0E20EF31E063071F786E390E01C
:108AD0000E94FA158EED91E00E942C182C018EEA6E
:108AE00099E00E942C18480E591E882499248EE97A
:108AF00099E00E942C185C01F401ED53F84F859128
:108B000094910E942C188C018AE999E00E942C18FB
:108B10006C01F401E35CF74F859194910E942C184D
:108B20007C0181E999E00E942C180A0D1B1D0C0D97
:108B30001D1D0E0D1F1D080F191F400E511E42E076
:108B400050E0840E951E5CE08516910481F680E06D
:108B500090E00E9458426091680570916905480E46
:108B6000591E88E1A2010DC657E0452E512C480C34
:108B7000591C002309F043C0D40117968C91882317
:108B800019F480E090E038C000E010E06E01089435
:108B9000C11CD11C46E0842E912C800E911EF40144
:108BA000E757FC4F65917491C2010E94A7627C0156
:108BB000009701F10396B6010E943F3E813079F49F
:108BC000F401ED56FC4F8591949101C0A895F99957
:108BD000FDCF49815A816B817C810E946463089436
:108BE000E108F108F701108202501040FFEF083F42
:108BF0001F0781F681E090E00E94DD44C4C501308A
:108C000009F081C0D2018C91882319F48824992419
:108C100059C0DE011C96EEE8F1E088E001900D926B
:108C20008150E1F732E1832E912C8C0E9D1E00E0E5
:108C300010E02CE3C22ED12CCC0EDD1E90E2B92E1A
:108C400086E0282E312C200E311EF101E750FC4F1A
:108C500065917491C2010E94A7627C01009779F12D
:108C6000F6012B2D11922A95E9F7BC016D5F7F4F1C
:108C7000C6010E940263D4018D919C91B6010E94AD
:108C80000263F101E75DFB4F6591749101C0A89506
:108C9000F999FDCFC60140E250E00E94426308947A
:108CA000E108F108F7011082025010402EEF3FEF6B
:108CB000820E931E3FEF083F130709F0C1CFB1E0CA
:108CC0008B2E912C81E00E94FA426C0180E00E9480
:108CD00053442C0181E00E9453447C0182E00E94B5
:108CE00053448C0183E00E9453444C0C5D1C4E0C99
:108CF0005F1C400E511E480E591E41E0841691041F
:108D000009F07FC07BC0023009F08FC0D2018C9186
:108D1000882319F48824992445C0C20167EC79E0BE
:108D20000E94A7627C010097D1F105960E94F63C53
:108D300090931B0880931A088F5F9F4F31F4109215
:108D40001B0810921A0801C0A895F999FDCF6091EF
:108D50001A0870911B0884EC90E00E9470630894DC
:108D6000E108F108F7011082C20164EC79E00E9489
:108D7000A7620097A1F00396BE016F5F7F4F0E942C
:108D80003F3E813061F401C0A895F999FDCF49813A
:108D90005A816B817C8180EC90E00E946463A1E049
:108DA0008A2E912C82E00E94FA426C0184E00E949B
:108DB0008D442C018CEC99E00E942C187C018E01D2
:108DC0000C5E1F4F80911A0890911B08B8010E94F9
:108DD000513CF80101900020E9F73197E01BF10BBD
:108DE000C801BF010E945F154C0C5D1C4E0C5F1C3E
:108DF000480E591EF1E08F16910419F48DE093E0AE
:108E000002C085E493E00E942C187C01E40CF51C60
:108E100081E090E00E945842609168057091690578
:108E2000E80EF91E88E1A701ACC4033009F04FC178
:108E3000C2010E943142813019F4F8E0FF2E05C0D2
:108E4000823011F40E949A4FFF2483E00E94D142A5
:108E50008C0189E39AE00E942C186091680570915A
:108E60006905080F191F88E1A8010E94AA2288231A
:108E700009F089C486E390E00E94FA156F2CAA24B9
:108E8000BB24ECE22E2E312C2C0E3D1E2F2D285F04
:108E9000C656DF4F2883CA59D040E62DF0E074E073
:108EA000EE0FFF1F7A95E1F7DE015C96E050F64F7A
:108EB00080E101900D928150E1F7DBA04C8C5D8C3C
:108EC0003E8DCE57DF4F3883C258D0404F8DCF579D
:108ED000DF4F4883C158D04058A1C058DF4F588356
:108EE000C058D04079A0CAA08CA09DA08EA19FA1FF
:108EF000C258DF4F99838883CE57D04080E19BE0F2
:108F00000E942C188C016394862D0E9475437C016D
:108F100086E09BE00E942C18E00EF11EE80EF91E80
:108F20008D2D81508330D8F45E824D82CE57DF4F35
:108F30009881C258D0409F83CF57DF4FA881C15836
:108F4000D040A887C058DF4FB881C058D040B987FB
:108F50007A86CB86CE0105960E948A4304C08FEFA5
:108F60009AE00E942C18E80EF91E85EF9AE00E9404
:108F70002C182701480E591EE2E0DE1661F486EE39
:108F80009AE00E942C187C0189ED9AE00E942C182E
:108F9000E80EF91E77C0F1E0DF1609F06EC021E996
:108FA00082162EE7920644F08CEC9AE00E942C1870
:108FB0007C01E40CF51C5AC097FC02C08BE201C096
:108FC0008DE20E942815C40197FE03C090958195FB
:108FD0009F4FB1010E94513CF10101900020E9F73F
:108FE0003197E219F309C101BF010E945F154C01DD
:108FF00087EC9AE00E942C186C01C258DF4F488120
:109000005981CE57D04057FD02C08BE201C08DE29E
:109010000E942815C258DF4F88819981CE57D040D1
:1090200097FF03C0909581959F4FB1010E94513CDD
:10903000F10101900020E9F7E219F3093397CE011D
:109040008E96BF010E945F158C0183EC9AE00E940E
:109050002C1862E0E62EF12CE40CF51CE80CF91C4F
:10906000EC0CFD1CE00EF11EE80EF91E80EB9AE000
:109070000E942C18E80EF91E07C080EA9AE00E94B0
:109080002C187C01E40CF51C85E99AE00E942C1850
:10909000E80EF91EAE0CBF1CC656DF4F5881CA59E8
:1090A000D040651609F0F9CE6091680570916905A8
:1090B00088E1A5010E94AA22882309F064C386E3FF
:1090C00090E00E94FA1583E060E070E098C10430FF
:1090D00009F09DC1C2010E943142813039F488E01B
:1090E000C856DF4F8883C859D0400DC0823019F46C
:1090F0000E948F4F03C0833009F4179AC856DF4F80
:109100001882C859D04084E00E94D1428C0188E383
:109110009BE00E942C186091680570916905080F0A
:10912000191F88E1A8010E94AA22882309F02BC3F5
:1091300086E390E00E94FA15C956DF4F1882C7599E
:10914000D040EE961FAE1EAEEE9754E1252E312C88
:109150002C0E3D1E8EEC9BE00E942C188C01C956F3
:10916000DF4FE881C759D040C856DF4F9881C859B2
:10917000D040E90FF0E044E0EE0FFF1F4A95E1F721
:10918000CF018050954FDC011C962D913D914D9162
:109190005C911F97CD56DF4F288339834A835B83C9
:1091A000C359D0401A96CC901A971B96BC91C756BB
:1091B000DF4FB883C959D040DF01A85FB44FEC90AE
:1091C0001196DC90DC0116966C91169715965C91C1
:1091D000DF01AC5FB44F7C91DC0113964C91139787
:1091E000EE5FF44FE0812D913C9111971796FC9022
:1091F000FF2009F4CAC08F2D8150843028F48AEBF7
:109200009BE00E942C180BC03E832D83EF83488780
:1092100079875A876B87CE0105960E948A43080F8B
:10922000191F80EB9BE00E942C182C01EF2DF0E021
:10923000EE0FFF1FEC5BF84F859194910E942C1864
:10924000400E511E480E591EB5E0FB1609F03FC0F6
:109250008AEA9BE00E942C183C018E2D9D2DB101C5
:109260000E94BD3BF10101900020E9F73197E2191E
:10927000F309C101BF010E945F154C0184EA9BE024
:109280000E942C185C018C2DC756DF4F9881C9595C
:10929000D040B1010E94BD3BF10101900020E9F7EF
:1092A0003197E219F309C101BF010E945F156C01FA
:1092B0008DE99BE00E942C187C01CD56DF4F888100
:1092C0009981C359D040B1010E94BD3B41C0EAE041
:1092D000FE1621F0F7E0FF1609F05EC086E99BE07C
:1092E0000E942C183C018E2DB1010E94A53BF1017A
:1092F00001900020E9F73197E219F309C101BF019C
:109300000E945F154C018FE89BE00E942C185C01C5
:109310008C2DB1010E94A53BF10101900020E9F7DD
:109320003197E219F309C101BF010E945F156C0179
:1093300087E89BE00E942C187C01CD56DF4F6881A6
:1093400079818A819B81C359D040A1010E94E73B6A
:10935000F10101900020E9F73197E219F309C10109
:10936000BF010E945F158C0189E20E9428150894B4
:10937000411C511C460C571C480C591C4A0C5B1CC8
:109380004C0C5D1C4E0C5F1C05C081E79BE00E94ED
:109390002C182C01400E511E86E69BE00E942C18D2
:1093A000480E591EEE962EAD3FADEE97240D351D9D
:1093B000EE963FAF2EAFEE97C956DF4F3881C759B3
:1093C000D0403F5FC956DF4F3883C759D04038304F
:1093D00009F0C0CE609168057091690588E1EE964C
:1093E0004EAD5FADEE970E94AA22882309F0CBC153
:1093F00086E390E00E94FA1584E061E070E00E944C
:109400006F428C0181E090E00E94584298C1053083
:1094100009F09EC185E00E94D142CF56DF4F99836B
:109420008883C159D04086E99CE00E942C188C01A9
:1094300060912D0570912E0580912F05909130053A
:109440002CE3E22EF12CEC0EFD1EA7010E94A33EA0
:10945000BC018BE89CE00E943743CD57DF4F9983D6
:109460008883C358D0406091310570913205809156
:10947000330590913405A7010E94A33EBC018FE7FC
:109480009CE00E943743CB57DF4F99838883C558B0
:10949000D0406091350570913605809137059091E7
:1094A0003805A7010E94A33EBC018FE69CE00E9404
:1094B0003743C957DF4F99838883C758D04060919D
:1094C000E1097091E2098091E3099091E409A70113
:1094D0000E94A33EBC0184E69CE00E943743C7572C
:1094E000DF4F99838883C958D04087E59CE061EDC0
:1094F00079E00E943743C557DF4F99838883CB5863
:10950000D0408091E709E82FF0E0E770F070EE0FAF
:10951000FF1FEB55F74F65917491C7010E94896257
:1095200088E49CE0B7010E943743C357DF4F99831B
:109530008883CD58D04080917D01E82FF0E0EE0F78
:10954000FF1FEA58F64F65917491C7010E94896226
:109550008CE39CE0B7010E943743C157DF4F9983EA
:109560008883CF58D04080910001B7010E94A53B6D
:1095700080910101BE01625C7F4F0E94A53BB70153
:109580006C5F7F4F809102010E94A53B8DE2FE013E
:10959000EE5BFF4F8083B701695F7F4F80910301CE
:1095A0000E94A53BB701675F7F4F809104010E9435
:1095B000A53BB701655F7F4F809105010E94A53BE8
:1095C000FE01E75BFF4F108280E39CE0B7010E9441
:1095D00037431C0120919B04822F6AE00E94C561E1
:1095E000805D8CAF822F0E94C561905D9DAF1EAEE5
:1095F0008EE19CE0B7010E9437432C01C7016CE764
:1096000070E00E9489628DE09CE0B7010E943743C0
:109610003C018090F0099090F109A090F209B0907F
:10962000F309C501B4012CE330E040E050E00E94B2
:109630000762CA01B901A7010E94D03C7CE5C72E90
:10964000D12CCC0EDD1EB7016B5F7F4FC6010E948F
:109650000263C60167E07CE00E947562C501B40147
:109660002CE330E040E050E00E940762DC01CB01D7
:10967000B7010E94513CC601BE01615C7F4F0E9450
:10968000E362C60162E07CE00E94756283EF9BE0CA
:10969000B6010E9437436C0186EE9BE00E942C18B5
:1096A0007C0181E090E00E945842CF56DF4F488114
:1096B0005981C159D040040F151FCD57DF4FA881E4
:1096C000B981C358D0400A0F1B1FCB57DF4FE88129
:1096D000F981C558D0400E0F1F1FC957DF4F288191
:1096E0003981C758D040020F131FC757DF4F488139
:1096F0005981C958D040040F151FC557DF4FA881A5
:10970000B981CB58D0400A0F1B1FC357DF4FE881E8
:10971000F981CD58D0400E0F1F1FC157DF4F288150
:109720003981CF58D040020F131F020D131D040DB5
:10973000151D060D171D0C0D1D1D0E0D1F1D609115
:10974000680570916905080F191F88E1A80119C003
:10975000609168057091690511C0E23079F486E383
:1097600090E00E94FA158DE691E00E942C18AC0161
:10977000609168057091690588E103C081E140E06E
:1097800050E00E94AA22C656DF4FE2E10C943E62EE
:10979000682F88E046E753E10E94191A0895E82FE0
:1097A000F0E0EE0FFF1FE65CFF4E4591549180E024
:1097B00061E00E94191A0895E82FF0E0EE0FFF1FF4
:1097C000E357F04F4591549180E060E00E94191AF0
:1097D0000895A0E1B0E0EFEEFBE40C942C62E09081
:1097E000F009F090F1090091F2091091F309C80114
:1097F000B7012CE330E040E050E00E940762CA016C
:10980000B9016E010894C11CD11CA6010E94D03C74
:1098100080E061E0AE014A5F5F4F0E94291AC801F3
:10982000B7012CE330E040E050E00E940762DC0129
:10983000CB01B6010E94513C8AE061E0AE014C5F71
:109840005F4F0E94291A6096E8E00C944862A4E0F9
:10985000B0E0EDE2FCE40C942A62B82EA62E6A0178
:10986000FA0180817E010894E11CF11CB7010E947D
:10987000353C8E010E5F1F4F8B2D6A2DA8010E9473
:10988000291A8AE30E94C019F6018181B7010E945A
:10989000353CC8010E94C7198AE30E94C019F6012D
:1098A0008281B7010E94353CC8010E94C7192496E5
:1098B000EAE00C944662A3E0B0E0E1E6FCE40C943C
:1098C0002D62D82E7A018B0140348EE7580785E04F
:1098D000680780E0780738F088E06D2D4DE653E1A9
:1098E0000E94191A2EC0CB01BA0120E13EE040E0EF
:1098F00050E00E9407622983C801B70120E13EE0E1
:1099000040E050E00E940762162F072FF82EE92E44
:109910002CE330E040E050E00E9407622A83612F90
:10992000702F8F2D9E2D2CE330E040E050E00E9400
:1099300007626B8388E06D2DAE014F5F5F4F0E9421
:10994000274C2396E7E00C944962809158088130B7
:1099500049F4409151085091520860915308709118
:1099600054081BC08731E1F480914D0890914E0856
:10997000A0914F08B09150088F5F9F4FAF4FBF4FDE
:1099800019F4EAE7F0E115C0409145085091460806
:10999000609147087091480881E00E945B4C0895EF
:1099A000883119F4E8E7F0E104C0893139F4E6E7D9
:1099B000F0E14591549188E061E004C088E061E005
:1099C00046E753E10E94191A0895A3E2B0E0EBEED6
:1099D000FCE40C942962082F0E94E819093018F45D
:1099E000402F4F5C02C0402F49508FE060E00E9442
:1099F000341AE02FF0E044E0EE0FFF1F4A95E1F744
:109A0000DE011496E050F54F80E101900D928150F7
:109A1000E1F7DB849E81CF809884A984BA848D2D60
:109A20008150843068F18D2D8550823248F534E1C3
:109A3000E32EF12CEC0EFD1E892FB7010E94353C60
:109A40008E010B5E1F4F80E060E0A8010E94291A82
:109A50008FE20E94C0198C2DB7010E94353CC801CD
:109A60000E94C71980E20E94C0199982AA82BB8213
:109A700086E060E0AE014F5F5F4F0E94274C06C05A
:109A800080E060E042E553E10E94191AED2DF0E01C
:109A9000EE0FFF1FEC5FFC4E4591549180E061E0BA
:109AA0000E94191AA396EBE00C944562A3E2B0E081
:109AB000ECE5FDE40C942862182F0E94E8198BE075
:109AC0000E94DC4BE12FF0E064E0EE0FFF1F6A958F
:109AD000E1F7DE011496E050F64F80E101900D921F
:109AE0008150E1F7DB84CE80BF8088849984AA848A
:109AF00054E1E52EF12CEC0EFD1E812F8F5FB70196
:109B00000E94353C8E010B5E1F4F8EE060E0A80185
:109B10000E94291A80E061E00E94F0198D2D815089
:109B2000823068F58C2DB7010E94353CC8010E9437
:109B3000C7198FE20E94C0198B2DB7010E94353CD6
:109B4000C8010E94C71980E20E94C01989829A82C6
:109B5000AB8286E061E0AE014F5F5F4F0E94274C11
:109B600080E20E94C01982E0D81611F482E404C099
:109B700081E0D81651F482E50E94C01906C080E049
:109B800061E042E553E10E94191AA396ECE00C94BF
:109B90004462A3E1B0E0EFECFDE40C942662809116
:109BA000F509E82FF0E0EE0FFF1FEC56FF4E659130
:109BB0007491CE0108960E94896260901D01709098
:109BC0001F0180902101A0902901B0902A010091ED
:109BD0002501109126010F5F1F4F90902301809166
:109BE000270190912801FCE0CF2ED12CCC0EDD1E58
:109BF0008459984FB6010E94513CEDE0EE2EF12CB5
:109C0000EC0EFD1E80E060E0A7010E94291A8FE2A1
:109C10000E94C019802FB6010E94353CC7010E94E6
:109C2000C7198FE20E94C019892DB6010E94353CE8
:109C3000C7010E94C71980E20E94C0198E010C5F03
:109C40001F4FAA0CBB1CAA0CBB1C8FE59EE0A80EE4
:109C5000B91EC801B5010E948962C8010E94C719D6
:109C600080E20E94C0190091E709077091F4809189
:109C70000601803C11F481E415C0803411F489E4BC
:109C800011C0803811F484E40DC08091F407805D28
:109C900009C0013011F482E505C0023011F08AE4F8
:109CA00001C087E40E94C01989827A826B8280E0B9
:109CB00061E0AE014F5F5F4F0E94274C80E20E943F
:109CC000C019CE0108960E94C71980E20E94C019EF
:109CD000023060F480910701BE016C5F7F4F0E94EB
:109CE000353CCE0105960E94C71921C00230C9F447
:109CF0008091E709887321F486E40E94C0190FC09F
:109D0000883011F482E503C0803189F48AE50E942D
:109D1000C0198091E70986FF02C082E506C086E48B
:109D200004C080E30E94C01981E30E94C019E09141
:109D30007D01F0E0E558F14FE4918E2F0E94C019AB
:109D40006396EEE00C944262A0E1B0E0EAEAFEE441
:109D50000C942C620091E5090E94E819002319F483
:109D60000E94C94DD8C0013019F580E060E041E49F
:109D70000E94341A60912D0570912E0580912F0557
:109D8000909130058E010F5F1F4FA8010E94A33EE6
:109D90000E94C71980E061E04DE40E94341A60918E
:109DA000310570913205809133059091340524C0BE
:109DB000023041F580E060E047E40E94341A60918F
:109DC00035057091360580913705909138058E01E3
:109DD0000F5F1F4FA8010E94A33E0E94C71980E099
:109DE00061E044E40E94341A6091E1097091E20953
:109DF0008091E3099091E409A8010E94A33E0E948A
:109E0000C71989C0033079F581E00E94DC4B80914D
:109E10009B046AE00E94C561805D0E94C019809128
:109E20009B046AE00E94C561892F805D0E94C01971
:109E300083E00E94CF4B04E0B0E0EB2EB1E0FB2EBC
:109E40006E010894C11CD11CF70181917F01B601FC
:109E50000E94A53BAC01802F61E00E94291A0E5F91
:109E6000003191F758C0043061F480E060E041EDCA
:109E700059E00E94291A84E00E94CF4B0E94A54C11
:109E80004AC0053091F586E00E94DC4B8091E709DD
:109E90008770823031F0813021F08091F60988237B
:109EA00091F188E060E046E753E10E94191A85E0ED
:109EB0000E94CF4B80911A0890911B08892B71F05A
:109EC0008091F7099091F809019741F40E94840E5E
:109ED000AB01BC0181E00E945B4C1DC088E061E0E9
:109EE00046E753E10E94191A16C00630A1F48CE02F
:109EF0000E94DC4B85E061E041E653E10E94191AC3
:109F00000E94E94B08C00E949F0EAB01BC0180E09B
:109F10000E945B4CCCCF6096E8E00C94486280E0F5
:109F200091E0E0E0FBE0DF019C011D922150304018
:109F3000E1F7089580E091E0E0E0FAE0DF019C01C4
:109F40001D9221503040E1F70895EF92FF920F9358
:109F50001F93182F80E19BE060E07BE040EF50E032
:109F60000E94CA626091270170912801E091250149
:109F7000E0902301F090210100911F01F0911D015B
:109F8000153079F4409195045091960420919304F2
:109F9000309194048091910490919204A0E0B0E0FB
:109FA00032C01A3011F0173089F480913C05482FE7
:109FB00050E080913D05282F30E080913E05909142
:109FC0003F05A0914005B09141051DC0812F8850EB
:109FD000823048F080E090E0A0E0B0E020E030E0A7
:109FE00040E050E010C04091AE045091AF04209189
:109FF000AC043091AD048091A4049091A504A0918B
:10A00000A604B091A70480930C0B90930D0BA09322
:10A010000E0BB0930F0B30930B0B20930A0B509346
:10A02000090B4093080B1093070BF093060B00935A
:10A03000050BF092040BE092030BEF5FE093020B31
:10A040006459784F7093010B6093000B1A3079F0CC
:10A050001B3169F0113259F01C3049F01D3039F0D4
:10A06000113029F0123019F0143009F017981F91AF
:10A070000F91FF90EF900895FF920F931F93F82E8A
:10A0800080E19AE08C0100511040B80140EF50E0AF
:10A090000E94CA6280912701909128018459984FAB
:10A0A000509125015F5FB0912301A0912101F091B2
:10A0B0001F01E0911D016091F6077091F707209153
:10A0C000F8073091F9074091F50710920F0A1092A6
:10A0D0000E0A10920D0A40930C0AF092070A309370
:10A0E0000B0A20930A0A7093090A6093080AE09306
:10A0F000060AF093050AA093040AB093030A50934A
:10A10000020AF801918380831F910F91FF900895B7
:10A110001F93CF93DF93EC01162F1092140C1E8621
:10A120000C960E94F63C8E3391050CF066C090931D
:10A130006601809365011C86CE010A960E94F63C5A
:10A140008C3391050CF059C090936801809367019E
:10A150001A86CE0108960E94F63C883191050CF0D3
:10A160004CC090936A01809369011886CE010696CF
:10A170000E94F63C009709F440C080329105ECF54E
:10A1800090936C0180936B011E82CE0104960E9415
:10A19000F63C01978C30910584F590936E01809385
:10A1A0006D011C82CE010E94F63C8C569740909324
:10A1B000700180936F0110927201109271011092E0
:10A1C00074011092730185E691E00E94A81D6093CE
:10A1D0000E0C70930F0C8093100C9093110C8091C7
:10A1E0000E0C90910F0CA091100CB091110CB7FDBA
:10A1F00002C01093140C81E001C080E0DF91CF9188
:10A200001F910895AF92BF92CF92DF92EF92FF928B
:10A210000F931F93379B08C01092FA091092F90907
:10A2200089E080937D017AC180917D01893019F4A4
:10A2300082E080937D011091F609112309F46EC12B
:10A240001130D9F41092140C0E94FA1A8091F90975
:10A250009091FA09892B19F483EA93E102C08CE901
:10A2600093E10E94231C82E08093F6090E94C11AA8
:10A270009093FC098093FB0951C11230D9F50E94DB
:10A280000E1B813009F034C18091F9099091FA09CF
:10A29000892BC1F48AE094E066E973E145E050E07F
:10A2A0000E949962892B39F481E090E09093FA0939
:10A2B0008093F90911C080E490E00E94BC0E1093D5
:10A2C0007D0113C18AE094E06DE873E148E050E05D
:10A2D0000E949962892B11F483E052C0A1E4B1E09D
:10A2E000EDE1F1E082E101900D928150E1F71092F1
:10A2F000F60915C1133041F40E94FA1A86E893E179
:10A300000E94231C84E0B0CF143009F051C00E9499
:10A310000E1B813009F03FC01092140482E194E0DA
:10A320000E94F63C009779F18032910564F5909394
:10A330006C0180936B01109211048FE094E00E94F5
:10A34000F63C01978C309105F4F490936E01809364
:10A350006D0110920E048AE094E00E94F63C8C5647
:10A36000974097FD10C09093700180936F011092F9
:10A37000720110927101109274011092730185E0C4
:10A380008093F609CBC080E490E00E94BC0E81E08F
:10A3900080937D01AAC00E94C11A2091FB093091CF
:10A3A000FC09821B930B805D974008F4B7C0ABC0DB
:10A3B000153041F40E94FA1A8FE793E10E94231CA2
:10A3C00086E052CF163009F0A9C00E940E1B8130E2
:10A3D00009F08EC01092120480E194E00E94F63CD5
:10A3E0008C3391050CF081C09093660180936501D8
:10A3F00010920F048DE094E00E94F63C8C3391059E
:10A400000CF073C0909368018093670110920C0464
:10A410008AE094E00E94F63C883191050CF065C01A
:10A4200090936A018093690185E691E00E94A81DDE
:10A430007B018C0180E7A82E81E8B82E8FEFC82E13
:10A440008FEFD82EEA0CFB1C0C1D1D1D17FD48C0FC
:10A45000F8942091020C3091030C4091040C50911F
:10A46000050C789480911B0190911C01892B01F5BA
:10A4700080911F08909120080097D1F05701680142
:10A48000A21AB30AC40AD50AA6019501D7FE07C0CD
:10A4900050954095309521953F4F4F4F5F4FA0E02D
:10A4A000B0E082179307A407B50714F482E019C03F
:10A4B000E0920E0CF0920F0C0093100C1093110C04
:10A4C00081E08093140C1092F9071092F807109213
:10A4D000F7071092F60710927D0110927C0105C0DB
:10A4E00081E080937D010E94950B1092F60916C0C1
:10A4F0000E94C11A2091FB093091FC09821B930B29
:10A50000805D974058F080E490E00E94BC0E83E0AC
:10A5100080937D011092F60985E201C080E01F91D1
:10A520000F91FF90EF90DF90CF90BF90AF90089584
:10A53000A1E0B0E0EEE9F2E50C942862182F0E9449
:10A54000FA1A183019F48FEF93E106C0103111F0A8
:10A55000CC244BC08BEC93E10E94231C0E94C11AB7
:10A560005C018C01CC24DD244E010894811C911CDB
:10A5700002C0DD2487010E94C11A7C010817190757
:10A5800009F0A895C7018A199B09805D974018F0CA
:10A5900025E2C22E2AC0DD2059F4C4010E94DE1A31
:10A5A000813041F78981843229F7DD24D394E2CFC9
:10A5B00081E0D81669F40E940E1BC82E21E0821794
:10A5C00019F492E0D92ED6CF82E0C81699F60DC0C4
:10A5D00022E0D21679F68AE094E06DEB73E14DE06B
:10A5E00050E00E949962892B21F68C2D2196ECE097
:10A5F0000C944462FC01808191819A3239F09A3046
:10A6000029F03196992311F08927F6CF0E94A53BB6
:10A610000895A5E1B0E0EFE0F3E50C942E6280919F
:10A620008D0490918E04892BD1F4CE0101960E9465
:10A63000DE1A813009F0BCC18981843209F0B8C1C9
:10A640000E94C11A90938C0480938B0481E090E067
:10A6500090938E0480938D0410928A04A9C10E9465
:10A660000E1B813009F093C11091E709187309F0AE
:10A6700058C08AE094E062EB73E14AE050E00E9447
:10A680009962892B09F094C190911504993331F4A2
:10A6900081E3809313049093140406C082E38093B3
:10A6A000130480E38093140483E194E062E070E09B
:10A6B0000E948850813009F05CC1F8941092010C1E
:10A6C0001092000C80910E0C90910F0CA091100C28
:10A6D000B091110C80930E0890930F08A09310086E
:10A6E000B09311088093020C9093030CA093040C78
:10A6F000B093050C789480912204813311F484E0A6
:10A70000D5C0823321F485E080937D01D8C08333A6
:10A7100009F04EC180912404803309F030C186E0F5
:10A72000C5C08AE094E0BE016E5F7F4F0E94FA527E
:10A730008AE094E06AE270E00E94EE62FC0191819E
:10A740008A81981709F036C192818B81981709F098
:10A7500031C18AE094E066E971E044E050E00E9493
:10A760000963009731F48091E70980688093E709D5
:10A770001FC1183009F0A6C08CE094E06EEA73E1C6
:10A7800043E050E00E949962892B09F011C18AE0F0
:10A7900094E06CE270E00E94EE62009709F4C4C09D
:10A7A0008C010F5F1F4FCE010E96B80146E050E0BE
:10A7B0000E941763C8016CE270E00E94EE62FC0127
:10A7C000009709F4B1C0F18001966CE270E00E943C
:10A7D000EE62009709F4A8C001966CE270E00E9456
:10A7E000EE62009709F4A0C001966CE270E00E944E
:10A7F000EE62009709F498C001966CE270E00E9446
:10A80000EE62009709F490C001966CE270E00E943D
:10A81000EE62009709F488C001966CE270E00E9435
:10A82000EE62009709F480C001966CE270E00E942D
:10A83000EE628C01009709F477C0BC016F5F7F4F17
:10A84000CE010C9642E050E00E941763B8016D5FA4
:10A850007F4FCE010A9642E050E00E941763B80194
:10A860006B5F7F4FCE01089642E050E00E94176375
:10A87000F8018581873324F081E38E8389E303C067
:10A8800082E38E8380E38F83CE01069661E070E0E1
:10A890000E948850882309F46CC0F1E4FF1609F483
:10A8A0006AC026E5F21609F03FC088E080937D017A
:10A8B0008091EA099091EB09892B09F465C00E9407
:10A8C000950B76C0103109F073C08CE094E06AEA11
:10A8D00073E143E050E00E949962892B09F068C05F
:10A8E00088E080937D018AE094E06CE270E00E9451
:10A8F000EE620097B9F08C010F5F1F4F36E0E32E38
:10A90000F12CEC0EFD1ECE010E96B80146E050E093
:10A910000E941763C8016CE270E00E94EE628C0135
:10A92000009721F40E94950B83E245C00F5F1F4FF3
:10A93000CE010C96B80142E050E00E9417630D5F13
:10A940001F4FCE010A96B80142E050E00E94176303
:10A950000D5F1F4FC701B80144E050E00E9417632C
:10A96000C70161E070E00E948850882321F40E94B2
:10A97000950B82E220C08091130C882311F087E0B0
:10A9800001C086E080937D0110927C0111C00E947D
:10A99000C11A20918B0430918C04821B930B885E2A
:10A9A000934030F010928E0410928D0485E203C023
:10A9B00080E001C084E26596E6E00C944A62A8E07B
:10A9C000B0E0E5EEF4E50C942E6281E00E94131AEB
:10A9D00081E061E041EB56E10E94191A8091EA0999
:10A9E0009091EB097E010894E11CF11CB7010E94D3
:10A9F000513CAC0186E061E00E94291A86E061E0EA
:10AA0000A70125E000E010E00E94703F892B19F4B7
:10AA100021E030E012C0C7010E94F63CBC019093D7
:10AA2000EB098093EA0901C0A895F999FDCF82ED61
:10AA300090E00E94706320E030E0C9012896E6E0D3
:10AA40000C944A62A8E0B0E0E8E2F5E50C942E62CE
:10AA500081E00E94131A81E061E04FEB56E10E9411
:10AA6000191A8091E8099091E9097E010894E11C86
:10AA7000F11CB7010E94513CAC0186E061E00E94EC
:10AA8000291A86E061E0A70125E000E010E00E94BD
:10AA9000703F892B19F421E030E012C0C7010E94F9
:10AAA000F63CBC019093E9098093E80901C0A895A0
:10AAB000F999FDCF80ED90E00E94706320E030E0D6
:10AAC000C9012896E6E00C944A621F93182F0E9451
:10AAD000E819E12FF0E0EE0FFF1FEE5CFA4E459112
:10AAE000549180E060E00E94191A1F910895EF923E
:10AAF000FF921F93DF93CF930F92CDB7DEB78FE016
:10AB00000E94655510918F04E12FF0E0EE0FFF1FBA
:10AB1000EC57F94E4591549180E061E00E94191A7A
:10AB20007E010894E11CF11C812F67E0A7010E94BF
:10AB30004D3F182F8981893109F45CC0843109F0B7
:10AB400049C010938F048091E7098770823079F5AE
:10AB50001092C100112319F484E395E01DC0113057
:10AB600019F48AE992E018C0123019F48CE491E0EB
:10AB700013C0133019F485EA90E00EC0143019F4B4
:10AB800082E590E009C0153019F489E290E004C034
:10AB9000163031F48BE190E09093C5008093C400AF
:10ABA00088E98093C1008091C60001C0A895F999F9
:10ABB000FDCF86E090E00E943C63792F01C0A8950C
:10ABC000F999FDCF86E090E0612F0E94706320E04C
:10ABD00030E012C081E00E94131AE12FF0E0EE0F86
:10ABE000FF1FEC57F94E4591549180E061E00E94BF
:10ABF000191A9ACF21E030E0C9010F90CF91DF916F
:10AC00001F91FF90EF900895A8E0B0E0EAE0F6E52C
:10AC10000C942E628EE00E94655581E061E042E96D
:10AC200056E10E94191A80911F08909120087E0118
:10AC30000894E11CF11CB7010E94513CAC0187E073
:10AC400061E00E94291A87E061E0A70125E000E0A9
:10AC500010E00E94703F892B19F421E030E012C00F
:10AC6000C7010E94F63CBC019093200880931F0806
:10AC700001C0A895F999FDCF88EC90E00E9470631F
:10AC800020E030E0C9012896E6E00C944A62A8E092
:10AC9000B0E0EDE4F6E50C942E628DE00E9465557F
:10ACA00081E061E041EA56E10E94191A809118089A
:10ACB000909119087E010894E11CF11CB7010E94D3
:10ACC000513CAC0189E061E00E94291A89E061E011
:10ACD000A70125E000E010E00E94703F892B19F4E5
:10ACE00021E030E012C0C7010E94F63CBC01909305
:10ACF00019088093180801C0A895F999FDCF86EC32
:10AD000090E00E94706320E030E0C9012896E6E000
:10AD10000C944A62EF92FF921F93DF93CF930F92AE
:10AD2000CDB7DEB78CE00E9465558091E70990E0D1
:10AD300056E0969587955A95E1F7182F1170E12FF7
:10AD4000F0E0EE0FFF1FEF5EF94E4591549180E069
:10AD500061E00E94191A7E010894E11CF11C812F08
:10AD600062E0A7010E944D3F182F89818931A1F12E
:10AD7000843111F501C0A895F999FDCF8CE390E0DD
:10AD80000E943C632091E709112331F42F7B20932B
:10AD9000E709BC01677F07C020642093E709BC0175
:10ADA000686001C0A895F999FDCF8CE390E00E94FE
:10ADB000706320E030E012C081E00E94131AE12F9E
:10ADC000F0E0EE0FFF1FEF5EF94E4591549180E0E9
:10ADD00061E00E94191AC3CF21E030E0C9010F9051
:10ADE000CF91DF911F91FF90EF900895EF92FF9226
:10ADF0001F93DF93CF930F92CDB7DEB78BE00E9406
:10AE000065551091E7091695169516951770E12F5F
:10AE1000F0E0EE0FFF1FE950FA4E4591549180E0AB
:10AE200061E00E94191A7E010894E11CF11C812F37
:10AE300063E0A7010E944D3F182F8981893109F4F1
:10AE40003AC0843141F501C0A895F999FDCF8CE352
:10AE500090E00E943C63BC01687F8091E709877C99
:10AE6000112319F48093E7090DC0113029F488608B
:10AE70008093E709616006C080618093E7096260A2
:10AE800001C0A895F999FDCF8CE390E00E94706312
:10AE900020E030E012C081E00E94131AE12FF0E0C0
:10AEA000EE0FFF1FE950FA4E4591549180E061E0AA
:10AEB0000E94191ABCCF21E030E0C9010F90CF9158
:10AEC000DF911F91FF90EF900895CF92DF92FF9254
:10AED0000F931F93DF93CF930F92CDB7DEB788E028
:10AEE0000E946555F090F509EF2DF0E0EE0FFF1F81
:10AEF000E855FA4E4591549180E061E00E94191A9C
:10AF00006E010894C11CD11C8F2D66E0A6010E9421
:10AF10004D3FF82E8981893109F434C00F2D10E09E
:10AF2000843109F5F092F509F801EE0FFF1FEE0FDD
:10AF3000FF1FEC54FA4E85919591A591B4918093A1
:10AF4000770190937801A0937901B0937A0101C0C1
:10AF5000A895F999FDCF8CEC90E0B8010E94706340
:10AF600020E030E011C081E00E94131AF801EE0FDA
:10AF7000FF1FE855FA4E4591549180E061E00E9430
:10AF8000191AC2CF21E030E0C9010F90CF91DF91B3
:10AF90001F910F91FF90DF90CF900895CF92DF9295
:10AFA000FF920F931F93DF93CF930F92CDB7DEB72E
:10AFB00087E00E94655501C0A895F999FDCF8AECFC
:10AFC00090E00E943C638C01FF24F394F822EF2D63
:10AFD000F0E0EE0FFF1FEF5BF94E4591549180E0DA
:10AFE00061E00E94191A6E010894C11CD11C8F2DBA
:10AFF00062E0A6010E944D3FF82E8981893191F1CE
:10B00000843101F58091E709982F9770FF2031F482
:10B01000B8016E7F913061F4887F06C0B80161602D
:10B02000992331F4887F81608093E70901C0A89556
:10B03000F999FDCF7F778AEC90E00E94706320E061
:10B0400030E012C081E00E94131AEF2DF0E0EE0F05
:10B05000FF1FEF5BF94E4591549180E061E00E9443
:10B06000191AC5CF21E030E0C9010F90CF91DF91CF
:10B070001F910F91FF90DF90CF900895A8E0B0E06E
:10B08000E4E4F8E50C942E6286E00E94655580E0C9
:10B0900061E04DEC56E10E94191A80911A089091D6
:10B0A0001B087E010894E11CF11CB7010E94513C71
:10B0B000AC0189E061E00E94291A89E061E0A70102
:10B0C00025E000E010E00E94703F892B19F421E098
:10B0D00030E012C0C7010E94F63CBC0190931B08EF
:10B0E00080931A0801C0A895F999FDCF84EC90E0EF
:10B0F0000E94706320E030E0C9012896E6E00C94DD
:10B100004A62A4E1B0E0E7E8F8E50C942C626B0138
:10B110000E94655501C0A895F999FDCFC6010E940E
:10B12000366369837A838B839C8325E0E22EF12C3E
:10B13000EC0EFD1EA7010E94A33E81E061E0A70185
:10B140002FE000E010E00E94703F892B19F421E00D
:10B1500030E015C0C701BE016F5F7F4F0E943F3EC8
:10B16000813059F401C0A895F999FDCF49815A81E0
:10B170006B817C81C6010E94646320E030E0C901DC
:10B180006496E8E00C94486285E060EC70E00E9410
:10B190008158089583E06CE270E00E948158089520
:10B1A00082E068E270E00E948158089581E064E2E4
:10B1B00070E00E948158089580E060E270E00E9493
:10B1C00081580895CF92DF92FF920F931F93DF93E0
:10B1D000CF930F92CDB7DEB784E00E94655501C0D2
:10B1E000A895F999FDCF8CE090E00E943C638C011A
:10B1F000F12EFF1CFF24FF1CEF2DF0E0EE0FFF1FD0
:10B20000EC5DF94E4591549180E061E00E94191A7D
:10B210006E010894C11CD11C8F2D62E0A6010E9412
:10B220004D3FF82E8981893141F18431B1F4FF20FD
:10B2300029F410925808B8017F7706C08093580807
:10B24000B801706801C0A895F999FDCF8CE090E035
:10B250000E94706320E030E012C081E00E94131A67
:10B26000EF2DF0E0EE0FFF1FEC5DF94E459154918C
:10B2700080E061E00E94191ACFCF21E030E0C901DF
:10B280000F90CF91DF911F910F91FF90DF90CF90A2
:10B290000895A4E0B0E0EFE4F9E50C943162182FD2
:10B2A0000E94E81980E060E041EE56E10E94191A20
:10B2B000E12FFF27E7FDF095EE0FFF1FEE5CFA4E42
:10B2C0004591549180E061E00E94191A812F8F5FAF
:10B2D000BE016F5F7F4F0E94353C8BE060E0AE01A6
:10B2E0004E5F5F4F0E94291A8DE060E04DED56E100
:10B2F0000E94191A2496E3E00C944D62CF92DF92DB
:10B30000FF920F931F93DF93CF93CDB7DEB7A19733
:10B310000FB6F894DEBF0FBECDBFDE011296EBE98B
:10B32000F1E080E201900D928150E1F70E944959CD
:10B33000FF246E010894C11CD11C8F2D61E1A60170
:10B340000E944D3FF82E89818931C1F0843119F076
:10B3500000E010E00EC080E1F81681F0EF2DF0E083
:10B36000EE0FFF1FEC0DFD1D0180F281E02D099510
:10B370008C018F2D0E944959012BF9F280915808B8
:10B38000882309F045C010925A081092590880E2AB
:10B3900090E044E651E068EA70EC0E94FC1B609388
:10B3A0002D0570932E0580932F059093300584E230
:10B3B00090E040E05FEF6FEF7FEF0E94FC1B609337
:10B3C000310570933205809333059093340588E2FC
:10B3D00090E041E051E068EA70EC0E94FC1B609351
:10B3E00035057093360580933705909338058CE2C8
:10B3F00090E041E051E068EA70EC0E94FC1B609331
:10B40000E1097093E2098093E3099093E40917C07E
:10B410008431A9F481E090E090935A088093590810
:10B42000A8E0B1E0EDE1F1E082E101900D92815000
:10B43000E1F70E942128882311F00E94A54FA196D0
:10B440000FB6F894DEBF0FBECDBFCF91DF911F9135
:10B450000F91FF90DF90CF900895EF92FF920F939E
:10B46000DF93CF93CDB7DEB760970FB6F894DEBF0A
:10B470000FBECDBFA82F002309F461C07E01089440
:10B48000E11CF11C88E0F70111928A95E9F7298304
:10B490003A834B835C836D837E83AF83988780E29E
:10B4A000801BE82FFF27E7FDF09549815A816B81CA
:10B4B0007C81181684F019861A861B861C868827BC
:10B4C00099278E1B9F0B04C0440F551F661F771FC3
:10B4D0008A95D2F728C0202F332727FD3095DB012E
:10B4E000CA01022E04C0880F991FAA1FBB1F0A940D
:10B4F000D2F789879A87AB87BC8704C07695679512
:10B5000057954795EA95D2F78D819E81AF81B88591
:10B5100004C0880F991FAA1FBB1F2A95D2F7482B7A
:10B52000592B6A2B7B2B4D875E876F87788B2985FC
:10B530003A854B855C856D857E85AF8598898A2F98
:10B5400060960FB6F894DEBF0FBECDBFCF91DF91EE
:10B550000F91FF90EF900895EF92FF920F93DF937A
:10B56000CF93CDB7DEB760970FB6F894DEBF0FBEAE
:10B57000CDBFA82F002309F467C07E010894E11C09
:10B58000F11C88E0F70111928A95E9F729833A8343
:10B590004B835C836D837E83AF83988780E2801BBF
:10B5A0004D815E816F817885E82FFF27E7FDF0955B
:10B5B0001816B4F0DB01CA01BB0F880B982FDC0111
:10B5C0008D879E87AF87B88B882799278E1B9F0B07
:10B5D00004C075956795579547958A95D2F728C009
:10B5E000202F332727FD3095DB01CA01022E04C02E
:10B5F000B595A795979587950A94D2F78D879E87DD
:10B60000AF87B88B04C0440F551F661F771FEA959C
:10B61000D2F789819A81AB81BC8104C0B695A79588
:10B62000979587952A95D2F7482B592B6A2B7B2B18
:10B6300049875A876B877C8729853A854B855C8546
:10B640006D857E85AF8598898A2F60960FB6F894B0
:10B65000DEBF0FBECDBFCF91DF910F91FF90EF9076
:10B660000895AEE5B0E0E7E3FBE50C942262A8E0C4
:10B670004E010894811C911CF4016A2E11926A9467
:10B68000E9F729833A834B835C836D837E838F83C1
:10B690009887CE010996FC011192AA95E9F7A9862F
:10B6A000BA86CB86DC86ED86FE860F87188B2984CA
:10B6B0003A844B845C84ED84FE840F85188969800C
:10B6C0007A808B809C806DA67EA68FA698AA6D80BE
:10B6D0007E808F809884E114F1040105110509F042
:10B6E000B3C3621473048404950408F03DC100E000
:10B6F000201600E0300601E0400600E0500688F425
:10B700001FEF211631044104510439F030F048E0B4
:10B71000E42EF12C012D112D18C0EE24FF248701F9
:10B7200014C020E0221620E0320620E0420621E08C
:10B73000520630F038E1E32EF12C012D112D05C019
:10B7400020E1E22EF12C012D112DD201C1010E2C90
:10B7500004C0B695A795979587950A94D2F7855416
:10B760009E4FDC012C9180E290E0A0E0B0E08E19C9
:10B770009F09A00BB10B7C018D01E21AF1080109B0
:10B780001109E114F10401051105A1F10E2C04C009
:10B79000220C331C441C551C0A94D2F7A4019301BB
:10B7A0000E2C04C0220F331F441F551F0A94D2F7DA
:10B7B00080E290E08E199F096DA47EA48FA498A8C2
:10B7C00004C096948794779467948A95D2F7622AF6
:10B7D000732A842A952AADA4BEA4CFA4D8A804C0F5
:10B7E000AA0CBB1CCC1CDD1CEA94D2F7ADA6BEA6ED
:10B7F000CFA6D8AA6201EE24FF24CDAADEAAEFAA22
:10B80000F8AE920181012070307009AF1AAF2BAFF2
:10B810003CAFC401B301A70196010E94E5617B0121
:10B820008C01C401B3012DA93EA94FA958AD0E94B6
:10B83000E561C901DA013C014D01C401B30129AD43
:10B840003AAD4BAD5CAD0E94A6619B01AC01870196
:10B85000FF24EE24ADA4BEA4CFA4D8A8C601AA2775
:10B86000BB2757016801A82AB92ACA2ADB2AA216CF
:10B87000B306C406D506E0F408946108710881088F
:10B880009108A20CB31CC41CD51CA214B304C4049C
:10B89000D50470F0A216B306C406D50648F4089481
:10B8A0006108710881089108A20CB31CC41CD51C46
:10B8B000A21AB30AC40AD50AC601B5012DA93EA928
:10B8C0004FA958AD0E94E5617B018C01C601B5010D
:10B8D0002DA93EA94FA958AD0E94E561C901DA0121
:10B8E0005C016D01C601B50129AD3AAD4BAD5CAD52
:10B8F0000E94A6619B01AC018701FF24EE248DA567
:10B900009EA5AFA5B8A9A070B070E82AF92A0A2BA5
:10B910001B2BE216F30604071507C0F40894A108D0
:10B92000B108C108D108E20CF31C041D151DE21476
:10B93000F3040405150550F0E216F3060407150795
:10B9400028F40894A108B108C108D108D3019927A7
:10B95000882786017501E82AF92A0A2B1B2BE9AAF8
:10B96000FAAA0BAB1CABCFC421143104410451041F
:10B9700071F461E070E080E090E020E030E040E0D1
:10B9800050E00E94E561C901DA011C012D0100E0CF
:10B99000201600E0300601E0400600E0500688F482
:10B9A0001FEF211631044104510431F028F048E022
:10B9B00050E060E070E017C040E050E060E070E010
:10B9C00012C020E0221620E0320620E0420621E0EC
:10B9D000520628F048E150E060E070E004C040E129
:10B9E00050E060E070E0D201C101042E04C0B695C1
:10B9F000A795979587950A94D2F785549E4FDC01B9
:10BA00002C91E0E2EE2EF12C012D112DD801C70171
:10BA1000841B950BA60BB70B821B9109A109B109D9
:10BA20000097A105B10561F464015301A218B308A0
:10BA3000C408D50831E0632E712C812C912C1EC1D5
:10BA40006F968FAF6F97082E04C0220C331C441CD6
:10BA5000551C0A94D2F7EE2DE81B640153010E2EFB
:10BA600004C0D694C794B794A7940A94D2F7A401BB
:10BA700093016F960FAC6F9704C0220F331F441FC2
:10BA8000551F0A94D2F76DA47EA48FA498A80E2EF9
:10BA900004C096948794779467940A94D2F78401AB
:10BAA0007301E22AF32A042B152BE9A6FAA60BA7A9
:10BAB0001CA73201882499249201810120703070E2
:10BAC00021960CAF1DAF2EAF3FAF2197C601B50138
:10BAD000A40193010E94E5617B018C01C601B501BF
:10BAE000A40193010E94E561C901DA0125968CAF9A
:10BAF0009DAFAEAFBFAF2597BC01CD0121962CAD58
:10BB00003DAD4EAD5FAD21970E94A6619B01AC019A
:10BB10008701FF24EE24A9A4BAA4CBA4DCA4C60107
:10BB2000AA27BB275C016D01AE28BF28C02AD12AF5
:10BB3000A216B306C406D50660F525966CAD7DAD9C
:10BB40008EAD9FAD25976150704080409040259606
:10BB50006CAF7DAF8EAF9FAF2597A20CB31CC41CFA
:10BB6000D51CA214B304C404D50498F0A216B306DD
:10BB7000C406D50670F46150704080409040259610
:10BB80006CAF7DAF8EAF9FAF2597A20CB31CC41CCA
:10BB9000D51CA21AB30AC40AD50AC601B501A4016C
:10BBA00093010E94E5617B018C01C601B501A401EE
:10BBB00093010E94E561C901DA013C014D01C40114
:10BBC000B30121962CAD3DAD4EAD5FAD21970E94E6
:10BBD000A6619B01AC018701FF24EE2489A59AA5EB
:10BBE000ABA5BCA5A070B07057016801A82AB92AFE
:10BBF000CA2ADB2AA216B306C406D506E0F40894C6
:10BC00006108710881089108A20CB31CC41CD51CE2
:10BC1000A214B304C404D50470F0A216B306C4067B
:10BC2000D50648F408946108710881089108A20CAF
:10BC3000B31CC41CD51C8DA59EA5AFA5B8A96F9635
:10BC40000FAC6F9704C0880F991FAA1FBB1F0A94DF
:10BC5000D2F78DA79EA7AFA7B8ABA21AB30AC40AA2
:10BC6000D50A2596ECACFDAC0EAD1FAD2597D701DE
:10BC700099278827682A792A8A2A9B2A82012227DB
:10BC8000332729960CAF1DAF2EAF3FAF2997A201E6
:10BC90009101407050702D962CAF3DAF4EAF5FAF0D
:10BCA0002D97C601B50129962CAD3DAD4EAD5FADCA
:10BCB00029970E94E5617B018C01C601B501299697
:10BCC0002CAD3DAD4EAD5FAD29970E94E561C90138
:10BCD000DA0161968CAF9DAFAEAFBFAF6197BC018B
:10BCE000CD012D962CAD3DAD4EAD5FAD2D970E9493
:10BCF000A6619B01AC018701FF24EE24ADA4BEA484
:10BD0000CFA4D8A8C601AA27BB2757016801A82A33
:10BD1000B92ACA2ADB2AA216B306C406D50660F5DC
:10BD200061966CAD7DAD8EAD9FAD619761507040F9
:10BD30008040904061966CAF7DAF8EAF9FAF6197B2
:10BD4000A20CB31CC41CD51CA214B304C404D50497
:10BD500098F0A216B306C406D50670F46150704080
:10BD60008040904061966CAF7DAF8EAF9FAF619782
:10BD7000A20CB31CC41CD51CA21AB30AC40AD50A4F
:10BD8000C601B50129962CAD3DAD4EAD5FAD2997ED
:10BD90000E94E5617B018C01C601B50129962CAD9D
:10BDA0003DAD4EAD5FAD29970E94E561C901DA0155
:10BDB0005C016D01C601B5012D962CAD3DAD4EADBA
:10BDC0005FAD2D970E94A6619B01AC018701FF2406
:10BDD000EE248DA59EA5AFA5B8A9A070B070E82AE5
:10BDE000F92A0A2B1B2BE216F30604071507C0F4E9
:10BDF0000894A108B108C108D108E20CF31C041D85
:10BE0000151DE214F3040405150550F0E216F306BF
:10BE10000407150728F40894A108B108C108D1083F
:10BE20006196ECACFDAC0EAD1FAD6197D7019927C3
:10BE3000882796018501082B192B2A2B3B2B09AB50
:10BE40001AAB2BAB3CAB62C26E147F04800691062A
:10BE500008F451C220E0E21620E0F20621E00207D9
:10BE600020E0120788F43FEFE316F1040105110505
:10BE700031F028F048E050E060E070E017C040E0AA
:10BE800050E060E070E012C040E0E41640E0F406EC
:10BE900040E0040741E0140728F048E150E060E08A
:10BEA00070E004C040E150E060E070E0D801C701FC
:10BEB000042E04C0B695A795979587950A94D2F756
:10BEC00085549E4FDC012C9130E2A32EB12CC12C65
:10BED000D12CD601C501841B950BA60BB70B821B79
:10BEE0009109A109B1090097A105B10589F4E614EA
:10BEF000F7040805190508F4F2C16DA47EA48FA407
:10BF000098A8621473048404950408F0E8C1F3C18E
:10BF10006E968FAF6E97082E04C0EE0CFF1C001FAC
:10BF2000111F0A94D2F76A2D681BD201C101062E97
:10BF300004C0B695A795979587950A94D2F75C01AA
:10BF40006D01AE28BF28C02AD12AADA2BEA2CFA2C1
:10BF5000D8A6720161016E960FAC6E9704C0CC0C2E
:10BF6000DD1CEE1CFF1C0A94D2F7C9A2DAA2EBA2D8
:10BF7000FCA264015301062E04C0D694C794B79462
:10BF8000A7940A94D2F7D401C3016E960FAC6E97B2
:10BF900004C0880F991FAA1FBB1F0A94D2F7EDA4F3
:10BFA000FEA40FA518A904C016950795F794E79469
:10BFB0006A95D2F737014801682A792A8A2A9B2A8A
:10BFC0006D8E7E8E8F8E98A2EDA0FEA00FA118A57B
:10BFD0003801882499249801870120703070659673
:10BFE0000CAF1DAF2EAF3FAF6597C601B501A401E1
:10BFF00093010E94E5617B018C01C601B501A4019A
:10C0000093010E94E561C901DA011C012D01C20101
:10C01000B10165962CAD3DAD4EAD5FAD65970E940B
:10C02000A6619B01AC018701FF24EE24AD8CBE8C80
:10C03000CF8CD8A0C601AA27BB2757016801A82A20
:10C04000B92ACA2ADB2AA216B306C406D50600F509
:10C0500008942108310841085108EDA0FEA00FA165
:10C0600018A5AE0CBF1CC01ED11EAE14BF04C00666
:10C07000D10670F0A216B306C406D50648F408949B
:10C080002108310841085108AE0CBF1CC01ED11E4A
:10C09000A21AB30AC40AD50AC601B501A4019301C4
:10C0A0000E94E5617B018C01C601B501A4019301E9
:10C0B0000E94E561C901DA013C014D01C401B301EF
:10C0C00065962CAD3DAD4EAD5FAD65970E94A66106
:10C0D0009B01AC018701FF24EE248D8D9E8DAF8DD9
:10C0E000B8A1A070B07057016801A82AB92ACA2A5D
:10C0F000DB2AA216B306C406D50600F5089461082B
:10C100007108810891086DA17EA18FA198A5A60E46
:10C11000B71EC81ED91EA616B706C806D90670F0E7
:10C12000A216B306C406D50648F40894610871083F
:10C1300081089108A60EB71EC81ED91ED601C501DA
:10C14000821B930BA40BB50B898F9A8FAB8FBC8F7F
:10C15000D1019927882764015301A82AB92ACA2A3C
:10C16000DB2AA9AABAAACBAADCAA860175012FEFFD
:10C170003FEF40E050E0E222F32204231523A60122
:10C18000662777276D964CAF5DAF6EAF7FAF6D972B
:10C19000A9A0BAA0CBA0DCA06FEF7FEF80E090E079
:10C1A000A622B722C822D92289A19AA1ABA1BCA1FB
:10C1B0001D0144245524C801B701A60195010E9420
:10C1C000A66169966CAF7DAF8EAF9FAF6997C801CE
:10C1D000B701A20191010E94A6613B014C016D963D
:10C1E0006CAD7DAD8EAD9FAD6D97A60195010E94A2
:10C1F000A6617B018C016D966CAD7DAD8EAD9FAD62
:10C200006D97A20191010E94A6615B016C01A801DA
:10C210009701260D371D481D591D69966CAC7DACE4
:10C220008EAC9FAC6997C401AA27BB27280F391F82
:10C230004A1F5B1F2E153F054007510748F4E12CAC
:10C24000F12C61E0062F112DAE0CBF1CC01ED11EBB
:10C25000CA01AA27BB27BC01CD016A0D7B1D8C1D1D
:10C260009D1D698C7A8C8B8C9C8C66167706880653
:10C27000990640F1661577058805990509F043C0D0
:10C28000D9019927882769962CAD3DAD4EAD5FAD9C
:10C29000699740705070820F931FA41FB51F2DA582
:10C2A0003EA54FA558A96E960FAC6E9704C0220FFD
:10C2B000331F441F551F0A94D2F7281739074A071E
:10C2C0005B0708F509A91AA92BA93CA90150104040
:10C2D0002040304009AB1AAB2BAB3CAB14C06624FA
:10C2E0007724430121E030E040E050E029AB3AAB55
:10C2F0004BAB5CAB0BC066247724430119AA1AAA86
:10C300001BAA1CAA03C0662477244301FE01719670
:10C3100088E0DF011D928A95E9F7A9A8BAA8CBA801
:10C32000DCA8A98ABA8ACB8ADC8A6D8A7E8A8F8A3F
:10C33000988E29A93A894B895C89662D7E898F89D7
:10C34000988DC25ADF4FE2E10C943E62629FD001A9
:10C35000739FF001829FE00DF11D649FE00DF11DC0
:10C36000929FF00D839FF00D749FF00D659FF00D6F
:10C370009927729FB00DE11DF91F639FB00DE11D5C
:10C38000F91FBD01CF0111240895991B79E004C064
:10C39000991F961708F0961B881F7A95C9F7809504
:10C3A0000895AA1BBB1B51E107C0AA1FBB1FA617FC
:10C3B000B70710F0A61BB70B881F991F5A95A9F74E
:10C3C00080959095BC01CD010895A1E21A2EAA1B7B
:10C3D000BB1BFD010DC0AA1FBB1FEE1FFF1FA21735
:10C3E000B307E407F50720F0A21BB30BE40BF50B32
:10C3F000661F771F881F991F1A9469F760957095BB
:10C40000809590959B01AC01BD01CF01089597FBEC
:10C41000092E05260ED057FD04D0D7DF0AD0001C08
:10C4200038F450954095309521953F4F4F4F5F4FD1
:10C430000895F6F790958095709561957F4F8F4F91
:10C440009F4F08952F923F924F925F926F927F92EB
:10C450008F929F92AF92BF92CF92DF92EF92FF9214
:10C460000F931F93CF93DF93CDB7DEB7CA1BDB0BC0
:10C470000FB6F894DEBF0FBECDBF09942A88398865
:10C4800048885F846E847D848C849B84AA84B9846C
:10C49000C884DF80EE80FD800C811B81AA81B98178
:10C4A000CE0FD11D0FB6F894DEBF0FBECDBFED018C
:10C4B0000895911106C080538A5010F0865C06C022
:10C4C000089599278827089585FDFBCF80629111F3
:10C4D000F8CF81568A51E0F7089591110895815659
:10C4E0008A5108F4805285580895FB01DC010D90B3
:10C4F0000020E9F7119705900D920020E1F70895CB
:10C50000FB01DC018D91059080190110D9F3990B85
:10C510000895FB01DC0105900D920020E1F70895DC
:10C52000FC0105900020E9F7809590958E0F9F1FE4
:10C530000895FB01DC014150504030F08D91059091
:10C54000801919F40020B9F7881B990B0895FB0195
:10C5500055915523A9F0BF01DC014D9145174111BB
:10C56000E1F759F4CD010590002049F04D914015B7
:10C570004111C9F3FB014111EFCF81E090E0019738
:10C580000895FB01DC0102C001900D924150504022
:10C59000D8F708956817790768F4FB01DC01E40F08
:10C5A000F51FA40FB51F02C002900E9241505040DB
:10C5B000D8F708950C94C162DC0101C06D9341501D
:10C5C0005040E0F70895FB01DC010D900020E9F7F1
:10C5D000119701900D920020E1F70895FC018191DF
:10C5E000861721F08823D9F7992708953197CF012D
:10C5F0000895FB01DC018D91019080190110D9F3A0
:10C60000990B0895FB01DC0101900D920020E1F7E8
:10C610000895FB01DC014150504030F08D910190B4
:10C62000801919F40020B9F7881B990B0895FB01B4
:10C63000DC014150504048F001900D920020C9F7B4
:10C6400001C01D9241505040E0F70895DC01CB013C
:10C65000FC01F999FECF06C0F2BDE1BDF89A319612
:10C6600000B40D9241505040B8F70895A6E1B0E0F3
:10C6700044E050E00C942863A8E1B0E042E050E0D0
:10C680000C942863DC01A40FB51F4150504048F0C2
:10C69000CB01840F951F2E910E945363415050404F
:10C6A000D0F70895262FF999FECF92BD81BDF89A53
:10C6B000019700B4021639F01FBA20BD0FB6F894E6
:10C6C000FA9AF99A0FBE08950396272F0E94536392
:10C6D0000E945263252F0E945363242F0C945363AE
:10C6E0000196272F0E9453630C945263DC01CB0107
:10C6F00003C02D910E94816341505040D0F70895AE
:10C70000262FF999FECF1FBA92BD81BD20BD0FB66D
:10C71000F894FA9AF99A0FBE01960895242F0E9470
:10C720008163252F0E9481630C9496630E9480632D
:0AC73000272F0C948163F894FFCFCB
:10C73A00020000000000C010000000000900010013
:10C74A000000460000000000000006010000000092
:10C75A00000900010000004600000000000000007F
:10C76A000000000000010000004600000000000078
:10C77A00000000000009000100000046000000005F
:10C78A00000000000000000900010000004600004F
:10C79A00000000000000000000090001000000463F
:10C7AA0000000000000000907E0000C8040215CDC1
:10C7BA005B07E5559A15B53B121F331349057407F4
:10C7CA009407B407D407504D544B00DC58D658D0C0
:10C7DA0058CA58E258C4583E58CE5765572255DFB2
:10C7EA0054F6568A564756045677550001020203F4
:10C7FA0003030304040404040404040505050505ED
:10C80A0005050505050505050505050606060606C9
:10C81A0006060606060606060606060606060606AE
:10C82A000606060606060606060606070707070799
:10C83A00070707070707070707070707070707077E
:10C84A00070707070707070707070707070707076E
:10C85A00070707070707070707070707070707075E
:10C86A000707070707070707070707080808080849
:10C87A00080808080808080808080808080808082E
:10C88A00080808080808080808080808080808081E
:10C89A00080808080808080808080808080808080E
:10C8AA0008080808080808080808080808080808FE
:10C8BA0008080808080808080808080808080808EE
:10C8CA0008080808080808080808080808080808DE
:10C8DA0008080808080808080808080808080808CE
:0CC8EA00080808080808080808080800EA
:00000001FF
